:020000021000EC
:109000000040002011140200791402007B140200B9
:109010000000000000000000000000000000000050
:109020000000000000000000000000007D140200AD
:1090300000000000000000007F1402008114020004
:109040007D0F0200831402008314020083140200C7
:109050008314020000000000B9E50100831402003F
:10906000831402008314020083140200831402009C
:10907000831402008314020083140200831402008C
:1090800083140200AD9301008314020083140200D4
:109090006D94010083140200F9E2010083140200C0
:1090A000831402008314020000000000000000008E
:1090B00000000000000000000000000000000000B0
:1090C0000090010036DF704737DF704710B503248A
:1090D0000723144010D1094B1A604B1CDB009BB2D4
:1090E000D218074B1A60074B1C70074B1C70074BBC
:1090F0001880074B1980231C181C10BD302000203D
:10910000342000203B2000203A200020382000207E
:109110003C200020F0B54A4B87B002921A8801909B
:109120000E1C039309208A4200D287E004ABDF1DA6
:1091300000233B70434B04255B68DB05DB0D21D02E
:10914000103BD9B24AB2002A0DDA0F220A40083A7F
:109150003D4B92089200D21855680322114091406D
:109160002B1CCB4009E09208C03238499200555878
:10917000032213409340DD402B1CDBB29B09DDB280
:10918000012B0DD0381CFFF79DFF022801D172B6CC
:1091900007E0002805D000210A1C01F0EFF900E0EB
:1091A0001D1C2B4B2B4A19782B4B12881C78C9B2EB
:1091B000E4B20020944201D20134E0B288420CD0E3
:1091C0001C781B780021DBB2934201D20133D9B263
:1091D000214B1970012D03D112E0012D2DD01F4C10
:1091E00062B63878FFF770FF0223021C9A4303D05F
:1091F00000210A1C01F0C2F9184B04209C421DD02A
:10920000174F029A3B68E5005B191A60019A002A21
:1092100010D0002E0ED0039B111C1B88321C5C4307
:10922000104B1868001908F0B7F93B6800205D1969
:10923000AE8003E00020988000E0042007B0F0BD7D
:109240003820002000ED00E018ED00E000E100E033
:109250003A2000203C2000203B200020FFFF00009F
:10926000302000203420002038B5104C104D2378D9
:109270002A789A4219D00F49237822780888D2B2E6
:10928000DBB20021904201D90132D1B20A4A2170E9
:1092900010880A4A58431268DB001018084A1268FE
:1092A000D31899881B689847E1E738BD3A20002019
:1092B0003B2000203C2000203820002034200020CB
:1092C00030200020174B02205968C905C90D27D04E
:1092D0001039CBB25AB2002A0DDA0F221A40083ADE
:1092E000C24082401049521803210B408B40526803
:1092F000DA40131C09E0032092080C4BC0329200A4
:10930000D25801408140131CCB40DBB29B09DBB239
:109310000020012B04D0033B5A4253410220C01AC3
:109320007047C04600ED00E018ED00E000E100E00D
:1093300080221A4B9202DA67D2218022184B520205
:1093400089005A50C22189005A5001212F225960A8
:10935000101C0138C046C046C046C046C046C04684
:10936000C046C046C046C046C046C046F1D199601E
:1093700000230C49101C0B600138C046C046C04693
:10938000C046C046C046C046C046C046C046C046AD
:10939000C046F1D1044A13707047C04604E100E0B2
:1093A000001001404020002068200020F8B5002473
:1093B000234B5C649C64DC641C655C609C60214B9A
:1093C0001E68731C3BD0204A204B214FD358214AA2
:1093D00015685D1B2D022D0A24235E433B689B19F3
:1093E0005A68954217D3AD1AA4181B4A1E6A126810
:1093F000D96994469A696346002B08D0101CE0474F
:10940000002806D000210A1C01F0B8F801E0081C71
:109410009047731CE0D1114B114A197813788B4295
:1094200005D10133DBB2022B00D100231370137876
:109430000C4A9B009C5080220B4B52035A60F8BD93
:10944000FC100140582000200010014004050000DD
:1094500048200020402000204420002054200020EC
:109460005520002060200020FCE100E0F0B5BD4A5E
:10947000BD491368BD488BB0029300780B789842C1
:1094800011D00133DBB2022B00D100230B700B781B
:10949000B7499B005B589C46029B63441B021B0A16
:1094A0001360012301E000239C460493B14B1B6829
:1094B0000593B14B1B780193B04B1B680993B04BDC
:1094C0001F681368019A0893AE4B00921B780393B0
:1094D000059B00990139CAB20092FF2A5FD0009A19
:1094E000D100099A51180C784A78A242F1D018227A
:1094F00062438D7801344868E4B22D1B8218681EDF
:10950000854110786D422C40022803D01D1C032891
:1095100043D139E0242052681D1C5043069238186C
:10952000027D0792002A38D01A1C6E1C08D0069EB5
:10953000B54207D024266E43BE192A1C356AF4E7CB
:109540001D1C1EE0AA4200D083E124256B43FB18BA
:109550001D6A6B1C06D101268B4B9E60079B0393F3
:1095600000230893242672434368BA180693036ABB
:1095700013625A1C05D07343FB185A68069E96194D
:109580005E600023037508E06B1C06D024235D4356
:1095900000237D192B752D6AF6E72B1CA4E769467D
:1095A000784A097B734C11706E4A089923601160E8
:1095B000049A002A09D1059A9B1A5A1E9341DBB2DC
:1095C000029301235B42009330E000206C4A242781
:1095D0001268051C03920122524200925A1C21D0AB
:1095E0003A1C5A4303998A1851688C4504D2236067
:1095F0006346C91A516017E06646761AB4464018A9
:109600001669116A556015750491002E08D00299EB
:10961000D66041180902090A91600099009311620D
:10962000049BDBE7534A136001230293514B1B68F1
:109630000393524B039A1B680693514B1B689C463D
:10964000484B1B6805934F4B1B780793019F013FC5
:10965000FBB20193FF2B00D19AE0019BD900069B3E
:109660005918131C009A013207D024220098424353
:109670006244041C106A009026E00A784878904200
:109680006ED0182050434C68013220188C78D2B22A
:109690000A70944201D100220A70027844681E1CAC
:1096A000012A5BD1242262436244157D002D55D1ED
:1096B00086689660C668D660066916614069D061A2
:1096C0000798002800D095609068059D2F4F451B96
:1096D0002D022D0AD668BD4202D8AD19556009E0A9
:1096E000059D281A0002000A864201D9301A00E0BE
:1096F0000020506000209060D0600120242510756B
:1097000001206543404210626544261C5A1C25D046
:1097100024225A43624468685668B04204D8301A1A
:109720005060261C2B6219E01A1C04932426564311
:1097300066447768B84206D9366AC01B0492771C23
:1097400005D0321CF2E73F1A7760161C049A686055
:1097500024202E621E1C424362441462331C81E7A3
:109760001A1C73E7402000205420002055200020C0
:1097700060200020582000204C2000205020002095
:10978000482000205C20002000100140FEFF7F00E8
:10979000314B1A60039B9A4202D1029B002B53D09B
:1097A000531C4FD024212D4B4A4318682C49821852
:1097B0002C4B2D481B680C5855682C4EE21A12028F
:1097C000120A3778033200920190002F20D18020B6
:1097D000D1274002BF00C851C127BF00C851C022D5
:1097E00080272348BF0252008750076001272F209F
:1097F0000F600138C046C046C046C046C046C0469D
:10980000C046C046C046C046C046C046F1D13770CB
:10981000009AAA4200D22A1CD318A8221B021B0AB3
:10982000D2008B50019A1B1B89581B02091B09028D
:10983000090A03311B0A994206D980220D4B920274
:109840005A6001E0FFF774FD00220B4B1A700BB059
:10985000F0BD1D1C86E6C046582000204820002090
:109860000010014040200020040500006820002076
:1098700000E100E0FCE100E05C200020F7B50325FA
:1098800001900F1C161C1C1C1D400720002D50D1E0
:10989000002B4ED0FFF74CFD264B089A1A60264B42
:1098A0001F70264B1C6024235F43E7193B1CA74213
:1098B00003D0257025752434F9E70321204A11705F
:1098C000204A00211760182218373C1C72435F6041
:1098D000197059709E7008330020BF18A342F6D14A
:1098E0000122194B52421A60184B80211870184BF4
:1098F000C5241870C023FF25164A49035B00D150C8
:10990000A4001359AB43C0252B431351A12311606D
:10991000019C1149DB00CC50C424A40015590F4B05
:109920002B40C0252D022B4313510D4BCA580D4B14
:109930001A60FEBD44200020562000204820002050
:109940004C200020502000205820002054200020CF
:109950005520002000E100E000100140FF00FFFF63
:109960000405000040200020F0B5104B061C1B68C9
:109970000820002B19D00720002A16D0002E14D062
:1099800000240B480778BC420EDA1D1C2433181C37
:1099900024380078002805D1012369702B70AA6152
:1099A000346002E00134EEE70420F0BD48200020DE
:1099B00056200020F7B5244B051C18680C1C082104
:1099C00000283FD0214B07211B789D423AD2042C1E
:1099D00038D924236B43C31818780821012831D1C2
:1099E0005B780027012B00D1271C161C0194FFF780
:1099F00069FC174BC0001A68121853789178581CEC
:109A0000411A4C1EA1414942084011788C4604215C
:109A1000604517D018214B435168CB180421002B07
:109A200010D001215D6019700A4D0B4969581F6102
:109A3000996001995E61D960507080220021074BC6
:109A400052035A60081CFEBD48200020562000200A
:109A5000502000200010014004050000FCE100E05F
:109A600038B51A4B041C1A680820002A2CD0184B51
:109A700007201B789C4227D2242363439B5C082049
:109A8000012B21D1FFF71EFC124BC0001B681B18D5
:109A90005D789A78691C8A1A501E824152421140A0
:109AA0001A78042091420FD018226A43586882180D
:109AB0000420002A08D00220546010708022002068
:109AC0005970054B52035A6038BDC04648200020EB
:109AD0005620002050200020FCE100E010B5041CBE
:109AE000082904D00020011C021C00F047FD60681A
:109AF0002368984710BD000007B5044A0090019103
:109B000068460821FFF706FB0EBDC046DD9A01003E
:109B10008023C0220349DB05D20099500021024A6C
:109B200099507047FFFFFF000406000029DF7047CF
:109B300028DF704737B5021C081C8B680D781C01A4
:109B40000B6949880830009102496458291CA047D4
:109B500037BDC04600220020F0B55C4C151C1A1C15
:109B6000237885B0071C002B06D12B1C134301D191
:109B7000022300E00123237023780320013B052BFF
:109B800000D9A0E0181C01920E1C07F0C7FC031EB0
:109B90002D6552868023E8205B0519691D691F69C0
:109BA0001B6989B28002019307F06CFC6B469A88AE
:109BB0000138ADB2B9B2684371439208FFF7B6FFFE
:109BC0000223002800D17DE07DE0081CFFF7B0FFF4
:109BD000002878D1002D2AD1019B002B23D13B787E
:109BE000042B1ED107231FE08022E82052051369B1
:109BF000116912699BB289B280025E43029207F03A
:109C000041FC6B461B89411E5943301C2A1CFFF73F
:109C10008DFF002857D1019B002B04D13B78042BEA
:109C200018D0052300E00423237000204BE0032319
:109C300048E080235B051B697A889BB25E43A800DD
:109C4000801939699208FFF771FF00283BD1019B09
:109C50001D43C7D00623E7E78022E8205205136999
:109C600079889BB202915E431169029B126989B2A5
:109C70008002F618039207F005FC6B469B890138B9
:109C80005843AD00029B76192D18E918301C019A33
:109C9000FFF74CFF0028C1D015E08023E8205B05CA
:109CA0001969800289B21D691E6907F0EBFBADB22C
:109CB0000138B1B2684307F0E5FBFFF739FF002830
:109CC00001D10723237005B0F0BDC0461922002042
:109CD000F7B514243C4B1A7854431C190092221CEB
:109CE00026790832271D95680193042E18D0052E79
:109CF0004AD00F20022E66D1344BE288188863695F
:109D0000800219182389121A5D19314B28189A42BA
:109D100001D8920801E080225200FFF707FF4DE0D2
:109D2000802651682B4A0B01D31818895A895B6821
:109D30007605AB4204D1131C4343E288934201D021
:109D400002290AD13169281C89B207F0C3FB1F4BD5
:109D50001B88C018FFF7ECFE30E03169281C89B27F
:109D600007F0B8FB14233269366992B24243011CF2
:109D7000B6B2013046430098AA1A434301989208AC
:109D8000C318DB88EB1814E0802676053169281C9F
:109D900089B207F09FFB3269366992B24243238948
:109DA000011CB6B201305B194643E0889A1A92084A
:109DB000C318F31A9B08381CFFF7CEFE002802D107
:109DC0000123019A9370FEBD6C2000201A2200200E
:109DD000FF03000000220020F8B5144D061C6C782B
:109DE00006A807880420142C1FD028782418E4B271
:109DF000132C01D9143CE4B2142044432C196261A1
:109E00000020221C267160710C3241C941C2E380DE
:109E10002781AB78002B01D0002003E0FFF758FF2B
:109E20001128F9D06B7801336B70F8BD6C200020DD
:109E3000F7B548498B780C1C002B00D189E0002530
:109E4000454B8D701A78082A07D1022800D0434B61
:109E50001D706378002B4BD17BE0022802D00328D1
:109E600052D076E00E7814213D4871430388611882
:109E700001339BB203800F790190022F04D1CA886D
:109E80009B02934210DA2DE0052F5BD0042F29D1DD
:109E9000C988D71F784278418C46071C9B02291C31
:109EA000634547DA002F4AD000232B4A1370019AEA
:109EB00013806378013B6370731CDBB2132B01D9F1
:109EC000331C133B237014235E43A619311D00205D
:109ED000FFF730FE002301213371F380F16033611D
:109EE000736133816378002B33D0A378002B30D19A
:109EF000FFF7EEFE00282CD011282AD01423217859
:109F000059436118043112E014230A780D20534399
:109F1000CB185A791C1D0132D2B25A71142A05D0BD
:109F2000FFF7D6FE002814D0112812D0211CFFF70D
:109F300001FE0EE00121002AB4D0291CB2E700295D
:109F4000D0D0B1E7D11F4A4251412F1C0029ABD1DB
:109F5000A8E7F7BD6C20002019220020182200205D
:109F60001A220020F7B500230120254A84461380D9
:109F70001A1C244C23706370A370A11D6546881EB3
:109F80000270E0180A80C560026142610281C82047
:109F9000143300260127143140008342EED180257E
:109FA000E820194B6D051E8029692B6989B2800252
:109FB000019307F067FA6B469B88023858430822E2
:109FC000124B1860E820124B80021E601E819E8199
:109FD0005E81104B1A7029692E6989B207F052FA16
:109FE0002D690138B6B2A9B2704307F04BFAFFF7FA
:109FF0009FFD002802D1084BA7701F70FEBDC04610
:10A000001A2200206C2000201022002014220020A0
:10A01000002200201922002018220020F0B5404B19
:10A0200087B01B780824002B76D00E24002873D02C
:10A03000002971D00368002B6ED0802783887F05AC
:10A0400000933E690724B6B2B34265D80F2B63D99B
:10A05000C388002B60D0334E051C3268E820019283
:10A06000009A03915A439446029239693B6989B236
:10A070000493019B80026344059307F003FA6B4647
:10A080001B8A01385843059B834245D83B69029A95
:10A090009BB29A4207DD3869009980B207F01AFA3C
:10A0A00089B2002938D10323009A07241A40131ECD
:10A0B00032D11D48042402880090012A2CD0039933
:10A0C00001980A60486019491401019F0819476006
:10A0D0002F688C4667508021AF8849050781ED883D
:10A0E00045817D4330680F690133BFB29BB2BD42E9
:10A0F00003D90F69BFB2ED1B00E0002580277F0563
:10A100003F69BFB2C019002DEDD16444A3812C1C5E
:10A11000009B013230601A80201C07B0F0BDC046A1
:10A1200018220020142200201022002000220020EB
:10A1300030B5104B1C780823002C19D00E230028B2
:10A1400016D0002A14D00368002B10D10A4D2C68B9
:10A15000002C0CD02C89406861430918688944435D
:10A1600068682418A14202D21360516000E00723FE
:10A17000181C30BD1822002000220020F7B5041C56
:10A18000194805780820002D2DD00E2000292AD04E
:10A19000002C28D025680720002D24D1134D2E68CF
:10A1A000002E20D066686F89B4462E896D6877438B
:10A1B0007F19BC4517D2002A15D0B24213D8D51842
:10A1C000B54210DC0325102029420CD12B420AD1C4
:10A1D00066462E4207D11D1C0220131C00950A1C46
:10A1E000211CFFF7F9FDFEBD1822002000220020EF
:10A1F000F7B5041C194805780820002D2DD00E2035
:10A2000000292AD0002C28D025680720002D24D131
:10A21000134D2E68002E20D066686F89B4462E89B3
:10A220006D6877437F19BC4517D2002A15D0B2421A
:10A2300013D8D518B54210DC0325102029420CD1C3
:10A240002B420AD166462E4207D11D1C0520131C45
:10A2500000950A1C211CFFF7BFFDFEBD182200203F
:10A2600000220020F0B50D1C111C244A85B0127884
:10A2700002930824002A3DD00E24002D3AD0002855
:10A2800038D02C68002C32D11D4E3268002A2ED0D6
:10A29000378973896A687B439C4673689C4462452E
:10A2A00025D2002923D0B94221D8029BCB18BB422A
:10A2B0001DDC03239C4618421BD1029F1F4218D16C
:10A2C0006746131C3B401F1E13D1029B0391991834
:10A2D000039A029007F060F9039A2B6800921B0121
:10A2E000F658281C03213A1C029BB04702E00724C1
:10A2F00000E01024201C05B0F0BDC046182200204C
:10A300000022002073B5154B041C1B780D1C08207F
:10A31000002B21D00E20002C1ED023680720002BFC
:10A320001AD10F4A1368002B16D05668118952892A
:10A3300063684A43921993420ED210209A070BD1B8
:10A34000981B07F0C7F807200A1E05D100910420CA
:10A35000211C2B1CFFF740FD76BDC04618220020B3
:10A3600000220020064B1A780823002A06D00E236C
:10A37000002803D0034B5B7803600023181C704750
:10A38000182200206C20002077DF704747DF7047DD
:10A3900011DF704713DF704713B50322041C5049C7
:10A3A00001A807F0F9F84F4B002C00D189E00022FA
:10A3B0001A70692C48D014D8612C2ED008D8422CA1
:10A3C00075D1494806F07AFF012006F03FFF74E09E
:10A3D000622C2FD0682C6AD1444806F06FFF4448A5
:10A3E00069E06C2C50D002D86B2C3CD05FE0722C12
:10A3F00056D0762C5BD13F4806F060FF3E4BD868C4
:10A4000006F05CFF3D4806F059FF3D4806F056FF58
:10A410003C4806F053FF3C484DE03C4806F04EFFF8
:10A420003B4B186806F062FF2E2006F02FFF394BD9
:10A43000186815E004F09EF9041C374806F03EFF4A
:10A44000201C06F063FF38E080243448640506F0E1
:10A4500035FF606E06F04AFF2E2006F017FF206ED3
:10A4600006F044FF29E02E4806F028FF2D4C237803
:10A47000002B01D02C4800E02C4806F01FFF0122E1
:10A4800023785340237018E0294806F017FF06F0A0
:10A490001FFC002802D1274806F010FF26480AE0DA
:10A4A00080220121254BD205D150254803E0201CF4
:10A4B00006F0ECFE234806F001FF01A806F0FEFEC0
:10A4C00013BD1A78002A01D1012202E0012A01D12C
:10A4D00002221A701B78022BEFD104F083FFECE705
:10A4E000CD1A020029220020F617020029180200C6
:10A4F0006A180200281902002032002033190200D5
:10A500003E1902004A1902004F190200D417020036
:10A51000A8000010A4000010DC170200B21802000E
:10A52000B818020008230020CB180200D618020039
:10A53000E0180200E7180200EC18020044050000D1
:10A54000F41802005819020070B50A4E04AC2578C0
:10A55000367805AC2478AE420AD1074D2D78A54255
:10A5600006D10C1C111C1A1C07F016F801232370CD
:10A5700070BDC04610230020BB24002070B5061C0F
:10A58000141C0D1C114806F099FE301C06F0AEFE9E
:10A590000F4806F093FE0F4806F090FE201C06F0D0
:10A5A0008DFE0D4806F08AFE281C06F0AFFE0B4B10
:10A5B0001E600B4B1D600B4B1C60BFF34F8F0A4A94
:10A5C0000A4BDA60BFF34F8FFEE7C0466319020003
:10A5D000CD1A020090190200941902001C320020CA
:10A5E00058320020143200200400FA0500ED00E08B
:10A5F00013B5144C2378002B0AD0134B1868FFF7BF
:10A600002FFA002803D000210A1CFFF7B7FF2070A3
:10A6100000220E4B191CD8331A600D4BD4311B7815
:10A620000A60012B0AD10B4B08211B786846009267
:10A63000019204F0FBFC04F0B5FE01E004F0D2FE50
:10A6400013BDC046C82400200C2300202C2200206B
:10A6500028220020BB24002038B5FFF799FE184DB2
:10A66000041E286002D000210A1C08E0E8208002B5
:10A67000FFF790FE2860002803D0211C221CFFF762
:10A680007DFF8021C0220F4BC90352009950012148
:10A690001A680D4C0B1C83401A4200D0E36701304E
:10A6A0002028F7D18022B121084BD205D150BFF329
:10A6B0004F8F074A074BDA60BFF34F8FFEE7C04664
:10A6C0001832002000E100E004E100E01C05000079
:10A6D0000400FA0500ED00E0F7B50025324B0095C7
:10A6E0001B780195AB425DD0304C231C221CD43327
:10A6F000D8321B6812689A420ED12D4C2378AB4297
:10A7000050D02C4B1868FFF7ABF9A84202D0291C97
:10A710002A1C36E0207045E00A22694653431A5D40
:10A720000A70E218D1798D4207D2281CEA18A218C3
:10A730005278684482700135F5E71F4B68461A78F5
:10A740001E4B08211B7804F071FC1D4E051E1CD108
:10A75000271CD4373B681421581C06F0BBFED834A4
:10A760002368013139608B421BD1114C2378002BB7
:10A7700017D0104B1868FFF773F9051E03D000219E
:10A780000A1CFFF7FBFE20700BE03368984208D0EC
:10A790000C4806F093FD281C06F0A8FD0A4806F0B8
:10A7A0008DFD3560F7BDC046282200202C220020F8
:10A7B000C82400200C23002010230020BB240020EC
:10A7C000B429002098190200CD1A020010B5104BD0
:10A7D0001B78022B1AD00478002C09D000200D4AD7
:10A7E000011CFEF797FC002810D000210A1C0BE08A
:10A7F0004378002B0AD0201C211C074AFEF78AFC54
:10A80000002803D0211C221CFFF7B8FE10BDC04653
:10A81000292200204D11020071110200F8B5037ABF
:10A82000041C002B1ED0C379042B1BD1FFF7E0FEC4
:10A830002378212B04D1514806F040FDFFF70CFF8F
:10A840004F4D504C022B05D14F4806F037FD0123E8
:10A850002B7005E04D4806F031FD01232B700023DD
:10A86000237088E0657A002D05D0494806F026FD62
:10A87000FFF7BEFE7FE0474B1B78002B22D0E37929
:10A88000012B78D16278082A06D1434A1378002B2D
:10A8900071D0013B13706EE00A2A0AD13F4806F0DE
:10A8A0000DFD3F4804F0B8FB002864D0291C2A1C89
:10A8B0005DE039490B78052B5DD8581C0870384984
:10A8C000CA5458E0374B1B78002B03D12E2006F0DA
:10A8D000DDFC1EE0344806F0F1FC207806F006FDB1
:10A8E000324806F0EBFCE07906F000FD304806F057
:10A8F000E5FC251CE3792A1B01359A4206DA202063
:10A9000006F0C4FC287806F0F1FCF3E7234806F0D3
:10A91000D5FC284F14213E1CD8363568681C06F03B
:10A92000D9FD3B1CD4331B680131994203D1224825
:10A9300006F0C4FC1FE00A225543211C781906F0DA
:10A940002BFE33681421581C06F0C4FD1B4D013149
:10A950002C783160002C0ED1F621194B4900186873
:10A96000221CFFF727F8002803D0211C221CFFF728
:10A9700005FE01232B7006F025FCF8BD9B19020093
:10A98000B8240020BE240020A7190200AE1902003E
:10A99000B5190200B9240020BA240020CD1A020003
:10A9A000C024002008230020C7190200D919020082
:10A9B000E51902002C220020F9190200C824002009
:10A9C0000C23002008B5031C0A1C0020191CFFF7EB
:10A9D000D5FD0000F8B52B4C061C00213822201CA8
:10A9E00006F01CFE284B01222360284B00256360E3
:10A9F000274B6283E360274BA5602383264B2561A9
:10AA0000A3820223A375E1182377244BCA77A3847A
:10AA100081235B00E385231C192130331D70231C27
:10AA20006185D22132331D70231CA185032131336E
:10AA30001970A2184B21D5770622194BE2841970A0
:10AA40004221102259709D70164B2285E577A5771B
:10AA5000657765631868144F391C06F0A9FE134B1F
:10AA600013486363211C231DDE77276104F0BEF9C0
:10AA7000104B1860A84203D0291C2A1CFFF77EFD4A
:10AA8000F8BDC04620320020FE1902000F1A020055
:10AA9000161A020018500000D1180000C10300006F
:10AAA00000200020A40000101C22002049A5010065
:10AAB000B9AA010018320020F7B5041C00780D284F
:10AAC00000D93DE106F034FD0E006500E0007000A5
:10AAD000D50099002C01AC00AE00B000C600CD003E
:10AAE0003501E9009B4F9C484C2101223B1C04F09E
:10AAF00043FC041E00D0B1E00823984E38780121B1
:10AB000000930196221C231C04F03AFC051E18D168
:10AB1000012338780093F318019302212A1C2B1C7F
:10AB200004F02EFC041E00D0D3E0022576193878FC
:10AB3000032100950196221C231C04F021FC00280F
:10AB400003D0211C221CFFF719FD03F013FE041C87
:10AB500004F0AAFA031C061CAB4308D0804806F098
:10AB6000ADFB301C06F0D2FB7E4806F0A7FB7E480A
:10AB700006F0A4FB201C06F0C9FB7C4806F09EFBF7
:10AB8000012004F09FFA002868D10420FFF7FCFBA5
:10AB9000DFE0774806F092FB96200122754BC0005B
:10ABA0001A7006F0B7FAD4E06379032B04D1724827
:10ABB00006F084FBA068C7E0022B00D0C9E06F4814
:10ABC00006F07CFBA06806F091FB6D4806F076FB72
:10ABD000A368187806F08AFB6A4806F06FFBA07934
:10ABE00006F084FB684806F069FBE07906F07EFB1E
:10ABF000664806F063FB2079A6E0654806F05EFB38
:10AC0000A08806F083FB634806F058FBE08806F056
:10AC10007DFB614806F052FB208906F077FB95E04A
:10AC20005E4894E05E4892E0302106225D4806F0DE
:10AC3000F5FC002005F07AFE01225B4B5B481A70A0
:10AC400000225B4B1A705B4B191CD833D4310A605D
:10AC50001A607CE0584806F031FB584800210A1C75
:10AC600071E7012005F062FE00224F4B54481A7034
:10AC70006DE0544806F022FB207906F037FB52487D
:10AC800006F01CFB60795FE0504806F017FB0022DD
:10AC9000384B1A7004F0A6FB5BE04D4806F00EFB43
:10ACA0004C4C2578002D0AD000254B4806F006FBB9
:10ACB00025704A4C2078FFF78DFE257049E0484BFF
:10ACC0001B78022B24D1FFF763FB464E041E306035
:10ACD00003D0201C291C2A1C35E7E8208002FFF73E
:10ACE00059FB3060002800D02BE78021C0223E4B6A
:10ACF000C9035200995001211A683C4C0B1C834037
:10AD00001A4200D0E36701302028F7D105F07AFD20
:10AD1000374806F0D3FA0020011C06F029FA18E0A3
:10AD2000344806F0CBFA04F05DFB0022294B1A7080
:10AD30000FE0314806F0C2FAFFF75AFCFFF78CFC2F
:10AD40002E4806F0BBFA207806F0D0FA074806F045
:10AD5000B5FAF7BD10230020941B0200BB2400208D
:10AD60001F1A0200261A0200321A0200CD1A02002F
:10AD7000471A0200282200204D1A0200561A02002B
:10AD80005F1A0200661A02006E1A0200741A0200AC
:10AD90007A1A0200911A0200A21A0200B91A0200DD
:10ADA000C01A0200C0240020B9240020D01A0200DA
:10ADB000BA2400202C220020E61A0200ADDE00009A
:10ADC000F41A0200071B0200F7190200111B02000F
:10ADD0001B1B0200B8240020261B0200BE240020FA
:10ADE000292200201832002000E100E004E100E008
:10ADF000381B0200441B02004E1B02005A1B0200BB
:10AE0000F0B58FB0FEF784FE8027AF230126DB006C
:10AE1000FF05FE50A02303214C4ADB0599504C4A04
:10AE20000C2099504B4A9950E7220221D2009950A8
:10AE30008021A1220903D20099501421464AFEF72D
:10AE400045F9051E02D000210A1C0BE0434B0B21E3
:10AE500000930A22424BFEF711FD041E04D0201C71
:10AE6000291C2A1CFFF78AFB301CFFF78FFA3D4D87
:10AE7000211C281CDC2206F0D1FB2B1C3A48D433C1
:10AE8000D835311C394A2C601C60FEF76DFD051E5B
:10AE90003CD10A2003F0D2FCFF208024021C1821A0
:10AEA0001C23009506F042FAE400314806F006FA49
:10AEB000385906F01BFA2F4806F000FA3B59301CAF
:10AEC0003B512D4905F0AAFE041EC8D105F038FDFE
:10AED0002A4806F0F3F9201CFFF77CFD284806F00D
:10AEE000EDF9284B03AD6B60274B281CAB600223A8
:10AEF0002B709623DB002B6203236B6220232349F4
:10AF00002C76AB6206F09AF8002802D0211C221C95
:10AF1000A8E77620FFF740FA6120FFF73DFA6220AC
:10AF2000FFF73AFA6C20FFF737FA194CFEF79CF955
:10AF3000281C06F091F9002805D02878FFF72CFA94
:10AF4000201C06F0BBF906F0EFF8EFE74C07000015
:10AF5000340700004407000014230020F99A010080
:10AF6000CC2400202C2200200C230020D9A6010094
:10AF70005F1B0200CD1A02001DA80100711B020018
:10AF80007E1B0200D90C02004DF60100CDA7010086
:10AF9000891B020072DF704779DF70477DDF7047E1
:10AFA00065DF7047F0B50024061C251C87B00C9F98
:10AFB00000933B7803910292019333889D423ADAE1
:10AFC0007368A9005918042205A806F0E5FA04AB35
:10AFD00005A8D91C0022FFF7E3FF002835D104ABF8
:10AFE000DB78029A934222D16242624102993B7815
:10AFF000520059188A181F2A1BDC002C07D16946F9
:10B000009A1C3A700133009A097BDBB2D15404AB2D
:10B01000DC1C3A78009B05A89A18211CFFF7C0FF9A
:10B02000002812D1237801243A78D3183B700135D7
:10B03000C3E70C2009E00020844206D03B78019A47
:10B04000013B9B1A0199009A535407B0F0BDF7B524
:10B05000089E171C00960222051C1C1CFFF7A2FF6D
:10B06000002806D10096281C391C1022231CFFF74B
:10B0700099FFFEBD0023F0B51370037889B0061C5C
:10B080000D1C141C002B03D1B378002B4BD029E0EE
:10B0900043780C201D2B00DD50E10E2704ABFF1878
:10B0A0001D23881C391C3B80FFF778FF002800D047
:10B0B00044E13378022B03D13B8809221D2B08D9A8
:10B0C0007378002B03D09BB208221D2B01D90822D4
:10B0D0003B88DBB2591C29706A70227802329B18B7
:10B0E0002370D1E723780C201B2B00DD26E10E27EF
:10B0F00004ABFF18381CFFF74FFF002800D01DE1FC
:10B1000023785A1C22700322EA5423785A1C227096
:10B110001922EA5423783A88EB181A70120A5A70E6
:10B12000237802332370F378002B0ED023785A1C37
:10B1300022700222EA5423785A1C22700122EA5417
:10B1400023789A182270F278EA547368002B12D090
:10B150001A7823780C201C2B00DDEFE0591C21709D
:10B160000221E9542378591C21700A21E9542378DB
:10B17000591C2170EA543389002B03D1338A002BE8
:10B1800016D00AE0301C00940830022106222B1C45
:10B19000FFF75DFF0028F1D0D0E0301C00941030A4
:10B1A000032107222B1CFFF752FF002800D0C5E027
:10B1B000338B002B0AD0301C009418301421152238
:10B1C0002B1CFFF744FF002800D0B7E0336A002BA8
:10B1D00049D022780C20049206321F2A00D9ADE013
:10B1E00019880720052900D8A8E0554A554F8A1824
:10B1F00092B2BA4200D8A1E05A880392052A00D838
:10B200009CE04F4FBC469444674602AA97819789B9
:10B21000BC464C4FBC4500D890E04B4FB94205D0DE
:10B22000039ABA4202D0914200D987E0049A049965
:10B230000132227005226A542278511C2170122199
:10B24000A95422781988AA181170090A5170227815
:10B250000232D2B222705B88AA1813701B0A537094
:10B26000237802332370776A002F29D03A79217826
:10B27000931C881CDBB2C3180C201F2B5EDC4B1CFC
:10B28000033223706A5423785A1C2270FF22EA5436
:10B2900023783A88EB181A70120A5A70237802330E
:10B2A000DBB22370BA88002A0AD0B96807200029C7
:10B2B00044D0E81806F070F9BA882378D3182370C0
:10B2C000331C2C3305931B78002B01D1002035E073
:10B2D000B36A002B31D000230493059B049A1B789A
:10B2E0009342F3D90C27049B22785F43B36A511C25
:10B2F000DF193B7921700333AB5423785A1C227039
:10B300001622EA5423783A88EB181A70120A5A70F7
:10B3100020780230C0B22070BA88002A09D0B968FB
:10B3200000290AD0281806F037F9BA882378D318EC
:10B330002370049B0133DBB2CEE7072009B0F0BDD8
:10B340007FF3FFFF7DF30000FFFF0000F0B593B037
:10B350006B466A469E1D0023D71D0D1C33703B7043
:10B36000984204D0C3785B070FD407201DE0041C6B
:10B37000002D03D0EB78002BF7D10EE02A1C31789A
:10B380003B78201CFFF706FE0FE002A9321CFFF7F6
:10B3900071FE02AC0028EBD007E03A1C281C0AA979
:10B3A000FFF768FE0AAA0028E9D013B0F0BDA0DFBD
:10B3B0007047A2DF7047A3DF7047A4DF7047A6DFA6
:10B3C000704713B50B88112B05D0502B07D0102BCD
:10B3D0001ED18B8801E001235B42438218E0037D8C
:10B3E000002B15D0CC884289944211D1CB8B022BF3
:10B3F0000ED10268002A0BD08B1CDB7F0131C97F84
:10B400001B020B43012101AC99432170211C904781
:10B4100013BD0000F0B50B680124036001235B42FB
:10B4200043820A7993B003745B4B0275071C021DBB
:10B430000D1C201C04A98C700B80FFF7B8FF011CA9
:10B44000061E00D0A4E03B7D002B0FD002AE0322ED
:10B45000301C06F0E3F8102306221C4334706B7B8B
:10B460007370B378934302221343B3700BAE301C56
:10B4700000211C2206F0D2F802203278012102437A
:10B4800010203B7D8243194009010A433270591E46
:10B490008B4100225B427260F260326102AA1A4064
:10B4A00000237261B3616A46012393753B4B00210F
:10B4B000938203A8032206F0B1F86A46AB7B06AC80
:10B4C0001373EB7B00215373937B06229343022279
:10B4D00013430822934310229343012293436A4665
:10B4E00093732B7B201CD370142206F097F805ABC6
:10B4F000069303AB6360012323810023638101234F
:10B50000A3816B4603332361311CB888BB1D221C09
:10B51000FFF74FFF061E3BD1AB68002B37D06A46C2
:10B52000012393751E4B311C938203A8032206F05E
:10B5300075F86A462B7CA968137300235373937BB9
:10B54000062293430222134308229343102293437B
:10B55000012293436A4601A8937301F099FB051CED
:10B56000311C1422201C06F059F83A1C05AB23604C
:10B5700003AB6360ADB201AB66812581A581236118
:10B58000F8880E32211CFFF716FF061C00E0F88138
:10B59000301C13B0F0BDC0460F180000192A00007F
:10B5A00008290000F0B589B06B46D971DF1D037C16
:10B5B000051C002499422ED002AE211C0822301C0A
:10B5C00006F02CF8012333803B78E9882B74688AD5
:10B5D000321C74807760FFF7F0FE041C011E1AD144
:10B5E0006A8A0E4B08249A4215D02B7D002B12D06C
:10B5F00004AC201C102206F011F8EB88211C2380DB
:10B600000123A3707388A660A3807368E360688ACF
:10B61000FFF7D5FE041C201C09B0F0BDFFFF0000A1
:10B6200075DF704776DF70477ADF70477BDF7047E2
:10B63000F7B52E4B18882E4B984256D02D4A2E4CDB
:10B6400013780133DBB21370217B99422DD32B4940
:10B65000FFF7E6FF051C2A4F2A4E002D45D0A369AF
:10B66000002B42D0112D09D1274805F027FE27488D
:10B670000021274AFEF778F9051CEEE7381C05F093
:10B680001DFE1C4B187805F031FE301C05F016FE2F
:10B69000204805F013FE281C05F028FE301C05F09C
:10B6A0000DFE281CA3699847D7E700231370237C5D
:10B6B000002B13D03B21FFF7B5FF051E0ED0A36969
:10B6C000002B0BD0144805F0F9FD281C05F00EFEE8
:10B6D0000C4805F0F3FD281CA36998476369002B0B
:10B6E00003D0002201A802709847F7BDE42900208A
:10B6F000FFFF0000C2290020C4290020E629002005
:10B70000F71B0200CD1A0200E01B0200E029002016
:10B7100031B60100071C02001D1C020037B5184B92
:10B72000184A5B881188184C184D99420CD85288D9
:10B730009A4209D36369002B03D0012201A8027049
:10B74000984700232B7037BD2B78002B05D06369F9
:10B75000002BF6D001A80022F1E70D4B1B78002B3F
:10B7600001D1616800E0A1680A4B00221868FEF769
:10B7700021F90028E5D0A369002BE1D1E1E7C0461B
:10B78000BA290020E6290020C4290020B829002079
:10B79000C2290020E0290020144938B5021C0B1CE6
:10B7A00032CA32C332CA32C31268114C1A60002244
:10B7B000104B01681A70201C914213D0082205F02A
:10B7C000EBFE201CFFF730FF00280ED101220021E4
:10B7D000094B52421A80094B094A0A481970FEF770
:10B7E000C3F802E0FFF722FFEEE738BDC4290020CE
:10B7F000E6290020B8290020E4290020C2290020E1
:10B8000031B60100E029002008B5024B1868FEF7A8
:10B8100027F908BDE029002010B50388112B19D0A5
:10B8200002D8102B05D043E0122B3AD0502B21D058
:10B830003EE0011C82881F4B16311A801E480822E8
:10B8400005F0AAFE00221D4B1A701D4BDB899342A6
:10B850002ED12BE00122174B52421A800022174BA7
:10B860001A70184B1868FEF7FBF8002820D0144B0C
:10B870009B6912E0124CC188E289914218D1C38BB6
:10B88000022B15D10130C37FDB070FD40D4B186895
:10B89000FEF7E6F800280BD0A369002B08D09847E4
:10B8A00006E0811D0822044805F076FEFFF736FF0A
:10B8B00010BDC046E4290020BA290020C22900207A
:10B8C000C4290020E029002037B5144C011C0822AF
:10B8D000201C05F061FE201CFFF7A6FE211C051EA2
:10B8E0001AD10F4B22885B889A4202D862889A420A
:10B8F0000AD201240B4B1C700B4B1888FFF790FEEB
:10B900000A4B051C1C7007E0094B5B69002B03D038
:10B91000012201A802709847281C3EBDE62900209C
:10B92000BA290020B8290020E4290020C2290020DB
:10B93000C4290020A0DF7047A2DF7047A5DF704751
:10B94000A6DF7047A8DF704763DF7047F0B50E24AD
:10B9500099B0002800D10DE1002900D10AE14B681F
:10B96000002B00D106E101235B420380029101908C
:10B970008249102208A805F00FFE0A21804B06AD6F
:10B980002B8004AB08A8C918FFF7DEFF041E00D007
:10B99000F0E0019B01201A1D291CFFF7CBFF041EBC
:10B9A00000D0E7E0AB78019A11AD9371211C1C2205
:10B9B000281C05F033FE04222B786C6013432B7097
:10B9C000019BEC602C616C61AC619B7904AA937360
:10B9D0006C4B05AF9381211C0322381C05F01EFE21
:10B9E000002301223B701023134306227B70BB7897
:10B9F0000CAE934302221343082293431022934335
:10BA00000122211C1343301C1422BB7005F006FEDA
:10BA100007AB0C931423B381019B3481748134618F
:10BA200077609888291C321C0833FFF785FF041EB5
:10BA300000D09FE0211C1C22281C05F0EFFD0822ED
:10BA40002B786C601343102213432B70019BEC6026
:10BA50002C616C61AC619B7904AA93734A4B211CE5
:10BA60009381381C032205F0D9FD00230F223B707F
:10BA70007B78211C9343012213430F221340102291
:10BA8000134306227B70BB78301C9343022213437E
:10BA90000822934310221343012213431422BB7044
:10BAA00005F0BCFD07AB0C931723B381019B3481D8
:10BAB0007481346177609888291C321C1033FFF739
:10BAC0003BFF041E56D1211C1C22281C05F0A6FD9C
:10BAD00002222B786C6013432B70019BEC602C616D
:10BAE0006C61AC619B7904AA9373284B211C9381F0
:10BAF000381C032205F092FD0F223B78211C934352
:10BB0000012213430F221340102213433B700023E2
:10BB100006227B70BB78301C934302221343082219
:10BB2000934310229343012213431422BB7005F068
:10BB300075FD07AB336002233381B381029B7481AF
:10BB40003361019B77609888291C321C2033FFF7F2
:10BB5000F3FE041E0ED1029B5B680393039A019BC4
:10BB60009A62029B9B68002B01D0019AD36201224A
:10BB7000074B1A70201C19B0F0BDC046341C0200DF
:10BB8000301500003215000031150000341500009A
:10BB9000EE290020F0B5051C87B00E20002D23D023
:10BBA0002C88124B08209C421ED0114B1B78002B76
:10BBB0001AD0104E1023717069468F1D032102ACFC
:10BBC0003980B27000211A1C201C337005F026FD4C
:10BBD0002B8A288823800123A3700023211CA380A3
:10BBE000A760E660FFF7ACFE07B0F0BDFFFF000006
:10BBF000EE290020F0290020F0B589B0002800D1FE
:10BC0000B0E0002900D1ADE0826A002A00D1A9E0AD
:10BC10000B88112B1AD004D8102B00D0A2E08B88EF
:10BC200016E00D1C041C502B02D0512B12D099E0B1
:10BC3000C9880389994200D094E0082304A90B70B5
:10BC4000EB8B20350B718D6090478BE001235B42BD
:10BC5000038087E08A79022A00D083E00A89038A78
:10BC60009A4200D07EE08B7A043B022B00D879E028
:10BC7000022301AE0021082204AF301C3B7005F006
:10BC8000CDFC02233380002373806B4673602088D1
:10BC9000A18A321CFFF752FE002804D0E36A002B71
:10BCA00005D0984703E06B461B78DB0707D4FE23DB
:10BCB0002088FF33391CBB80FFF744FE4CE0B8807E
:10BCC000391C2088FFF73EFE002845D1EB1CD97FA8
:10BCD000481E07283CD805F021FC040E1B1D1F211F
:10BCE0003423002333702B8C012B02D8201C01211C
:10BCF00008E0012308E0012333702A8C9A4203D81C
:10BD0000201C0221062225E023353371B5601AE09C
:10BD1000022317E0032315E0042313E0052311E0B9
:10BD20002B8C022B02D8201C082112E06B1DDB7F1C
:10BD30000435EA7F1B021343B3805A425341063352
:10BD400000E009233370A36A201C311C984709E0E6
:10BD5000201C0322FFF71EFF002803D0E36A002BFC
:10BD600000D0984709B0F0BDA0DF7047A2DF704750
:10BD7000F0B593B003900191171C0293002903D1F1
:10BD8000081C0A1CFEF7FAFB002F04D1381C391CD2
:10BD90003A1CFEF7F3FB0BAC201C00211C2205F023
:10BDA0003DFC02222378002513436A46012692892E
:10BDB000237004AB9A80291C181C03229E716560B5
:10BDC000E56025616561A56105F028FC029B04AA78
:10BDD0001B78291C1370029B5B78537093780622A2
:10BDE000934302221343E7221340B34304AA06AE4F
:10BDF0009370301C142205F011FC05AB069304ABC4
:10BE00007360019B211C3361054B321C1888189B01
:10BE100037817581B781FFF7A9FF13B0F0BDC04628
:10BE2000402A002010B5041C012086B0544B03A901
:10BE3000544A88700B80FFF797FF002800D09DE0E0
:10BE40002288002A03D12289002A16D00AE04E4B0C
:10BE50004E480093231C61683C33FFF789FF00289C
:10BE6000F1D08BE04A4B4B480093231CE1683C33F4
:10BE7000FFF77EFF002800D080E0228A002A09D048
:10BE8000454B46480093231C61693C33FFF770FF24
:10BE9000002873D1228B002A09D0414B41480093DE
:10BEA000231CE1693C33FFF763FF002866D1228C35
:10BEB000002A09D03C4B3D480093231C616A3C3367
:10BEC000FFF756FF002859D1228D002A09D0384BA0
:10BED00038480093231CE16A3C33FFF749FF0028F0
:10BEE0004CD1236B002B1AD01A7804A90A705A7807
:10BEF00031484A709A788A70DA78CA701A790A7169
:10BF00009B681A0A4B711B0CCB712C4B8A710093E6
:10BF1000231C08223C33FFF72BFF00282ED1636B34
:10BF2000002B03D1A06B00280CD127E019681A79E7
:10BF3000234B24480093231C3C33FFF719FF0028B0
:10BF4000F0D01BE0037804A90B7043881E4A4B70A5
:10BF50001B0A8B708388CB701B0A0B71C3881B482C
:10BF60004B711B0A8B71231C00923C330722FFF795
:10BF7000FFFE031C0020834200D0181C06B010BD39
:10BF80000A180000402A0020102A0020292A000058
:10BF9000002A0020242A0000302A0020252A000040
:10BFA000282A0020272A0000382A0020262A0000FC
:10BFB000F8290020282A0000232A0000082A00204F
:10BFC000182A00202A2A0000202A0020502A0000D7
:10BFD000A0DF7047A1DF7047A2DF7047A3DF704783
:10BFE000A4DF7047A6DF704765DF7047F0B50768CC
:10BFF00087B00C1C002F10D0111C0422061C01ADB0
:10C0000002A82A7005F0C8FAA38B301C2B81E38BA1
:10C0100020346B81EC60291CB84707B0F0BD0000EC
:10C02000F0B5022793B00BAC0E1C01900021201C30
:10C030001C2205F0F3FA237800253B4323700123EB
:10C0400002AA9372204B291C138103A80322656066
:10C05000E56025616561A56105F0E0FA331C3433C4
:10C060001B7802AA1371331C35331B783036537199
:10C0700006239279291C9A43E72317431F40012383
:10C080009F4302AB9F71338805AF3B701B0A7B70E7
:10C09000B3781422BB70F37806AEFB70301C05F049
:10C0A000BDFA04AB069303AB736004233381B38101
:10C0B000019B7581376118896733FF33211C321C5E
:10C0C000FFF78AFF13B0F0BD4A2A000070B5138B4A
:10C0D00086B0022B11D10568002D0ED00123032656
:10C0E000041C927E02A81340F31A042201AE33709E
:10C0F00005F052FA201C311CA84706B070BD0000A4
:10C10000F0B5102695B002931AAB019204CB0090C3
:10C110001B780D1C03930B78334211D005AC03221E
:10C12000201C002105F07AFA012306221E431A9BE7
:10C1300026701B786370A378934302221343A37085
:10C140000DAF00211C22381C05F068FA10222B7854
:10C1500000263B701340591E8B4105AA5B421A40D2
:10C1600001237A6104AA9373394B06AD9381311C84
:10C170000322281C7E60FE603E61BE6105F04EFA1F
:10C18000062201211A9B08AC5B78201C2B701A9B9D
:10C190009B786B70AB789343039A0A4002210B4360
:10C1A0000821D2008B431343102293430122311CF8
:10C1B00013431422AB7005F031FA07AB08936B46BA
:10C1C0009B88391CA381009B221C18881C9B2681FC
:10C1D000668126616560FFF7FFFE061E35D10123EB
:10C1E00004AA93731B4B311C9381281C032205F076
:10C1F00015FA06221A9B311C5B78201C2B701A9BA7
:10C200009B786B70AB7893430222134308229343CD
:10C2100010229343012293431422AB7005F0FEF9E0
:10C2200007AB029904A80893656000F031FD04ABE8
:10C2300023611C9B80B21A1C2081A08108321888BF
:10C24000211C6681FFF7CAFE061C301C15B0F0BD2C
:10C250004D2A000008290000F0B595B005AF161C66
:10C2600001900291381C00210322039305F0D6F9B6
:10C2700001221023134306223B7033780DAC7B70F0
:10C28000BB78201C93430222002113431C22BB7065
:10C2900005F0C4F90F22B17823780A40511E8A4173
:10C2A00002210B430821D2008B4313431022134376
:10C2B0002370012304AA9373131C6A460025128974
:10C2C000676106AF9A81291C381C03226560E5600E
:10C2D0002561A56105F0A2F906227378291C3B703F
:10C2E000B37808AE7B70BB78301C934302221343B3
:10C2F0000822934310229343012293431422BB70DC
:10C3000005F08CF907AB08930823B381019B211C2E
:10C310001888321C039B7760358175813561FFF782
:10C320005BFE15B0F0BD0000F0B50B8887B0112B97
:10C3300031D0041C112B02D8102B06D02FE1502B2A
:10C340002FD0512B00D1A6E029E1BB228B885200CF
:10C3500083524389002B00D121E16B46012701ADB7
:10C3600000210822281CDE1CDF7005F057F900238D
:10C370006B80BB232F806E605B00E05A61892A1CB2
:10C38000FFF72EFE002800D109E16368002B00D1E1
:10C3900005E1984703E10122BB2352425B00C252F0
:10C3A000FDE0B7204000CB88205A8A1D984213D167
:10C3B000138B012B00D0F2E02568002D00D1EEE0B8
:10C3C000937E002B02D0012B00D0E8E001AA13706D
:10C3D000201C01A9A847E2E06089984216D1138B7E
:10C3E000012B00D0DBE02368002B00D1D7E0927E48
:10C3F000002A04D0012A00D0D1E0062100E0052166
:10C4000001AA1170201C01A99847C8E0A92040008A
:10C41000205A984202D101A9624B12E0A7204000A5
:10C42000205A984206D15F4B01AA138000239370D3
:10C43000D3701DE0B1204000205A984209D15A4BD8
:10C4400001A90B8000238B70CB70201CFFF73EFEF0
:10C45000A5E0AF204000255A00209D4203D0251CB6
:10C46000A67C183508E0504B01AA13809070D0705C
:10C47000201C83E00130C0B2B0423FD00A352F1CEF
:10C480000A3F3F889F42F5D1484B01A90B80012309
:10C49000C8708B70D9E78A79012A00D07FE0251C0B
:10C4A00000220889A67C1435D3B2B34206D22F8865
:10C4B00001320A35B842F7D1012262E0231C251C63
:10C4C000002278331E787A35D3B2B34206D22F8851
:10C4D00001320A35B842F7D1022252E0231C251C52
:10C4E0000022DE331E78E035D3B2B34257D22F8814
:10C4F00001320A35B842F7D1032242E0221C002063
:10C500001432B0420DD00A32151C0A3D2D889D42CE
:10C5100004D1264A01AB1A8001222BE00130C0B2BF
:10C52000EFE7221C0020783215780232A8420DD0A5
:10C530000A32161C0A3E36889E4204D11B4A01ABC1
:10C540001A80022216E00130C0B2EFE7221CDE3270
:10C5500015780020023201E00130C0B2A8421ED09E
:10C560000A32161C0A3E36889E42F5D10F4A01ABAC
:10C570001A800322D870201C9A7001AAFFF736FD9A
:10C580000DE02668002E0AD0072001AD287007486C
:10C59000AA71A880EB71201C0591291CB04707B037
:10C5A000F0BDC046222A0000332A00004D2A0000B8
:10C5B0000722F0B58B7A9DB004920A2B00D9AEE227
:10C5C0000B7C0A2B00D9AAE20B7E0A2B00D9A6E22B
:10C5D0000A68059002604A680D1C42608B7A837479
:10C5E000031C0A7C78331A700A7E66331A700122A3
:10C5F000BB2352425B00C2520120CE4B0AA90B80E2
:10C60000059B887008331A1C0693FFF7E1FC049021
:10C61000061E00D083E22B1C36331B7815ACB342C8
:10C620000DD9059BAA6B18897300995A221CFFF734
:10C63000D1FC002800D04DE10136F6B2EBE7002333
:10C6400004932B7A002B06D16B7A002B03D1AB7AA3
:10C65000002B4AD183E000211C220226201C04F07A
:10C66000DDFF042223782221334313432370012367
:10C67000002704AA52181370AF4B04AA1384391C64
:10C6800003220BA86760E76027616761A76104F078
:10C69000C5FF2B1C3C331A7804A90A775B788A7F84
:10C6A0004B7706239A43E72316431E4001239E43FC
:10C6B0008E7710AE391C1422301C04F0AFFF01221B
:10C6C00009AB1A700CAA10920BAA72600122336196
:10C6D000059B3281B28177811889211C321C0A3373
:10C6E000FFF77AFCB842B2D0F4E00026EB68B34220
:10C6F00035D0AB7AB34232D915AFEB6800210122B5
:10C70000F400381C1C1904F089FF02223B780598BC
:10C7100013433B700F23A2791A40511E8A4108210E
:10C720003B78D2008B431343102213433B70211DEF
:10C7300022880091E179A31CC907C90FC9B20191F0
:10C740000A2171434118143102910698391CFFF7F0
:10C75000D7FC002800D0BDE00136F6B2C9E72B7C3B
:10C76000002B04D000266B69B34200D0D8E02B7EAA
:10C77000002B00D0D8E0022615AC00211C22201C82
:10C7800004F04CFF2378002733432370012304AACD
:10C7900093776A4B391C938309A803226760E7608B
:10C7A00027616761A76104F039FF2B1C2C331B78CC
:10C7B00004AA13752B1C2D331B78391C53750623C3
:10C7C000927D9A43E72316431E4001231E4304AB88
:10C7D0009E7510AE1422301C04F020FF0BAB10939A
:10C7E00009AB7360AB8C77813381B3812B6A211CD9
:10C7F0003361059B321C18894533FF33FFF7ECFB8F
:10C80000B84200D011E1EB1DDB7F002B00D1C1E06D
:10C81000AB6A061C002B00D109E1EB1DDB7F9E42B9
:10C8200000DAB9E02B7A002B00D007E16B7A002BFD
:10C8300000D064E10598291CFFF7F2FB0490002862
:10C8400000D06CE115AC04991C22201C04F0E6FE1B
:10C85000042223780127134322222370049B0BAE6A
:10C860006360E36023616361A36104AB9B181F7085
:10C87000334B04AA138404990322301C04F0CEFE27
:10C8800006223E352B78022133706B7810AD737021
:10C89000B378281C9343E7220B4313406A46BB43FB
:10C8A000127CB37004AB1A750499142204F0B6FE1E
:10C8B0000CAB10936B461B8A6E606B8109AB2B61CE
:10C8C000059B2F81AF8118896F33FF33211C2A1CF0
:10C8D000FFF782FB049022E115AF6B690021012272
:10C8E000F400381C1C1904F099FE0E233A78211D1F
:10C8F00013433B7022880091E1790598C907C90F5D
:10C90000C9B201910A21714341187A310291A31CE5
:10C910000698391CFFF7F4FB0028DBD10136F6B28C
:10C920002B7CB342D8D822E70026EB69B3422DD145
:10C9300021E7C046121800004E2A00004B2A0000D2
:10C940004C2A000015AFEB6900210122F400381CCD
:10C950001C1904F063FE0A233A78211D13433B702F
:10C9600022880091E1790598C907C90FC9B20191E0
:10C970000A217143E03141180291A31C0698391C29
:10C98000FFF7BEFB0028A5D10136F6B22B7EB342DD
:10C99000D8D8F0E61E1C40E7012404AB9C77614B1D
:10C9A00009AF04AA938300210322381C04F036FE49
:10C9B000202323433B70002306227B70BB78022197
:10C9C0009343E7220B431340A343BB70AB6AB00011
:10C9D0001818132304AA9B18191C0CAAFFF704FBB0
:10C9E0000790031E1ED110AC191C1422201C04F049
:10C9F00015FE0BAB109304ABDB7C6A462381A3814D
:10CA00000CAB2361A223928B67606281059A5B0065
:10CA1000D05A4D32211CFF32FFF7E0FA002804D132
:10CA20000136FAE6079B049303E0049001E0072334
:10CA300074E0049B002B00D1F4E670E02A1C059BF7
:10CA400006984F33FF3338494332FFF705FC079010
:10CA5000031E62D115AC191C1C220226201C04F0F6
:10CA6000DDFD08222378222133431343042213439C
:10CA70002370049B04AA6360E36023616361A36184
:10CA8000012352181370294B0BAF04AA1384079982
:10CA90000322381C04F0C2FD2B1C46331B780622EF
:10CAA0003B702B1C47331B7807997B70BB789343F3
:10CAB0001E4308239E4310239E4301239E43BE70C2
:10CAC00010AE1422301C04F0A9FD0CAB10936B4681
:10CAD0001B8A776033816B461B8A211C738101237B
:10CAE000B381049B321C3361059B18895733FF3394
:10CAF000FFF772FA0490002800D197E60FE02A1C95
:10CB0000059B06985F330A494032FF33FFF7A4FBC9
:10CB10000490002800D18DE601E0079B049304985F
:10CB20001DB0F0BD07290000222A0000322A0000B3
:10CB3000332A0000F0B589B000920193837C051C74
:10CB40000F1C07208B422AD9BB235B00EA5A154BE6
:10CB500008209A4223D002AB9E1D6B4604AC1B8872
:10CB60000021201C1022338004F058FD0A235F436B
:10CB7000EF19BB8A211C23800123A3700023A3800B
:10CB8000019BA660E360BB235B00E85AFFF72AFA2B
:10CB9000002804D13388009A934200D00C2009B0B9
:10CBA000F0BDC046FFFF0000BB23F0B589B05B00BD
:10CBB0000192C25A134B061C0F1C08209A421FD028
:10CBC00004AC02ABD980201C002110229D1D04F072
:10CBD00025FDA7235B00F35A211C23800123A370AA
:10CBE0000023A380019BA560E360BB235B00F05A98
:10CBF000FFF7F8F9002803D12B88BB4200D00C20A6
:10CC000009B0F0BDFFFF0000F0B5071CBB204000DD
:10CC10008BB03E5A1D4D141C10AA12880820AE423B
:10CC200032D0D01C01906846858802A8861D3580C8
:10CC30000C20082D28D804AD29706C70AB70002A28
:10CC400005D00B2002ABC018119904F0A5FC06AC6E
:10CC50000021201C102204F0E1FCAF235B00FB5AF2
:10CC6000A66023800123A3700023A380BB23E5607B
:10CC70005B00F85A211CFFF7B5F9002804D133886E
:10CC8000019A934200D00C200BB0F0BDFFFF0000D2
:10CC90000B7803704B7843700220704738B5041C42
:10CCA000081C0D1C04F006FD6560208038BD7FDF88
:10CCB000704782DF7047A7DF7047A9DF7047AADFA0
:10CCC0007047002070470020704700207047002008
:10CCD0007047002070470020704700207047000018
:10CCE000F0B585B0041C0F1C02AA81782248FDF71C
:10CCF0001FFA00283ED10C236678204A5E4395191E
:10CD0000AB7A01925B0605D4022F03D0012F03D02A
:10CD10001B4D02E01B4D00E01B4D1C26A1781B4B58
:10CD2000714302A85918321C0023A847002813D1C8
:10CD3000022F1FD00C234021627802A85343019A8E
:10CD4000D3189A7A8A439A726178114B7143321CD4
:10CD50005918331CA84701E0022F0BD00C2322786E
:10CD600002A853430B4A211CD3189B7A0A4A9B0002
:10CD70009B58984705B0F0BD0C2B0020562A002088
:10CD8000C3CC0100F1A101007DA10100642A0020B3
:10CD9000B82A0020FC2A0020441C0200F7B52822F3
:10CDA0000190437829485A4381184C68284F002C39
:10CDB0000FD00C2159437918897A4DB2002D07DA2A
:10CDC000490605D4151C0835A6B24519145802E0C9
:10CDD0000024261C251C0C225343FB181889291CEF
:10CDE000321C231CFFF769FF0B2818D10C22019B72
:10CDF000291C5B785343FB181889321C0123FFF769
:10CE00005CFF00280ED00C21019B124A5B784B433B
:10CE1000FF183889FFF74FFF00280AD115E00028D6
:10CE200003D100E00124002000E00B48012C0CD1CC
:10CE3000E9E70222094BC318934303D0082801D025
:10CE4000112801D1044800E00020FEBDD42A0020B2
:10CE5000562A0020FFFF000041800000FECFFFFFA8
:10CE600008B5FFF79BFF08BD2023F0B58DB002AADF
:10CE7000D3800C2201904B780E1C5343254A04A901
:10CE8000D318188902AB9A1D0323FFF718FF002857
:10CE90003CD128247078204F604302AB0830DA88F8
:10CEA000381804A904F04EFB3D1C737800280DD1FE
:10CEB0000C225A4317498A18917A0222114025D12F
:10CEC0006343221CF81804F0A9FB1FE05C433C19E3
:10CED0006268002A01D1114F00E0114F282403227B
:10CEE0006343EA5002ABDA88737804A96343EB1812
:10CEF0005A60707860430830281804F04DFB717850
:10CF000001986143221C69183823B84700200DB0EE
:10CF1000F0BDC046562A0020D42A00207DA1010081
:10CF2000F1A1010008B5FFF79FFF08BD70B52824E7
:10CF3000031C4878094D60430E1C2818191C221C3C
:10CF40003823FDF78FF9002806D173785C432C193C
:10CF50006368013300D1606070BDC046D42A0020F0
:10CF600008B5FFF7E3FF08BDF0B5504C95B0256854
:10CF70000294002D00D197E01A9C782C00D993E000
:10CF80000024161CFF221D1C05AB5A709A70DA7023
:10CF90001C701A9B08AF019103903C700D950C9387
:10CFA000A1B2434806AAFDF7C3F8002809D10398A7
:10CFB00006A9082204F0C6FA002802D105AB9C702D
:10CFC00002E00134032CEBD105ACA378FF2B6BD02E
:10CFD000019908AA042907D11A9B782B01D1202393
:10CFE00000E04023137045E03249691A532910D8F4
:10CFF0003149002E04D1012098400D68054253D0DC
:10D0000001209840031C086898432023086013708F
:10D010003EE02A49691A1B2908D8202313700023EF
:10D0200063700EAB0D9318230C9331E02448291A3A
:10D0300027290ED830233B70002363700123E3704F
:10D04000204B997A0223194022D1282204F0E6FAD3
:10D050001EE0402111701C4A95420BD01B4A9900DA
:10D060008A58AA4220D1174AD27A9A4210D1002374
:10D0700063700DE0032108AA13780B4313700BAB08
:10D080000993029B201C1B6808A9321C98470BE0DF
:10D09000019A08AB032A02D11A78012101E002218A
:10D0A0001A780A431A70EAE715B0F0BDFC2A00208E
:10D0B0000C2B0020642A0020082B0020B82A002016
:10D0C000D42A0020562A0020741C0200442A002082
:10D0D00070B51C2444430F4E051C3019002134192F
:10D0E0000622113004F09AFA201C0021102204F0CC
:10D0F00095FAFF232374A37601235B422383012344
:10D10000AB40054AAD001168994311600022034B02
:10D11000EA5070BD642A0020082B0020442A002019
:10D1200037B581B2051C6A460748FDF701F8041EB1
:10D1300008D168467821FDF7E5F8041E02D1281CC5
:10D14000FFF7C6FF201C3EBD0C2B0020F0B585B0BC
:10D1500000285CD00127002601252E4B041C2E48F8
:10D160007F421E605E729E72311C0781C772072269
:10D17000857204F053FA311C2822284804F04EFA34
:10D18000301CFFF7A5FFFF23254E281C3370FFF747
:10D190009FFF02207770FFF79BFF78236A469380FA
:10D1A0000323B7701F4FD3801F4B6846391C009371
:10D1B000FCF734FF00282BD11C4B24781D701D1C5C
:10D1C000002C1AD11A4FA1B2164802AAFCF7B0FFE0
:10D1D000061E0BD11C22101C604302A93818331CF8
:10D1E000FDF740F8002804D02E7011E000232B70CA
:10D1F0000EE00134032CE6D10AE06B466A46DB8878
:10D200009188381C594389B2FDF77CF800E0094841
:10D2100005B0F0BDFC2A0020562A0020D42A0020A8
:10D22000502A00200C2B002069CF0100542A002036
:10D23000642A00200E800000F8B5174B1B78002BE5
:10D2400024D0002824D0002922D00B68002B1FD026
:10D25000124D2C68002C1DD1061C281C0F1C08C068
:10D260000531052204F098F90120022104223B79BE
:10D27000AB722B7A83430B4393432B72EB790343BB
:10D280000B439343EB71201C347004E0044802E02C
:10D29000044800E00448F8BD542A0020FC2A00207D
:10D2A000088000000E80000004800000F0B5254BCF
:10D2B0001B78002B25D0002821D000291FD00B6817
:10D2C000002B1CD08B68002B19D00378002B18D1B1
:10D2D0001D4A1268002A14D01A1C1C1C1B481C4D25
:10D2E000EF7ABB420FD1AF7A02252F420BD0013328
:10D2F0001C30032BF3D10C710A73002020E0154879
:10D300001EE015481CE00F7BBA4209D20125877E3A
:10D310002F4205D18D6897007851104DAB540132E2
:10D320000F79BC42E3D20225877E2F42DFD1102540
:10D33000AC46844466460D68A7007E510134D6E7AA
:10D34000F0BDC046542A0020FC2A0020642A002098
:10D35000562A00200E80000008800000502A00207D
:10D3600008B50A4B1B78002B0ED000280AD0037892
:10D37000002B09D1064B1B68002B05D08078FFF7E6
:10D38000CFFE02E0034800E0034808BD542A002015
:10D39000FC2A00200E8000000880000038B5104BE9
:10D3A0001B78002B19D0002815D00478002C14D13C
:10D3B0000C4B1B68002B10D0201C0B4D1C2363430F
:10D3C000EB189B7EFF2B02D0201CFFF7A9FE013437
:10D3D000032CF3D102E0054800E0054838BDC04603
:10D3E000542A0020FC2A0020642A00200E8000001D
:10D3F0000880000037B5214B1B78002B3AD000285D
:10D4000036D0002934D00378002B33D11C4B1B6855
:10D41000002B2FD04378002B2ED11A4B9B7A012B57
:10D420002AD08278022A27D81C235343164AD318BD
:10D430009B7EFF2B20D00C1CC968051C00290AD03C
:10D44000A268531E1E2B06D82378012B03D10F4848
:10D45000083004F0A1F8A9786A460D48FCF768FE88
:10D4600023780C4A9B009B586846291C984704E087
:10D47000094802E0094800E009483EBD542A00205E
:10D48000FC2A0020562A0020642A0020D42A0020EA
:10D490000C2B0020441C02000E80000008800000BD
:10D4A000108000007FB5294B051C1B78002B48D04D
:10D4B000002844D0002942D08B68002B3FD003784D
:10D4C000002B3ED1224B1B68002B3AD08378022BD5
:10D4D00039D81C225A431F488218927EFF2A32D024
:10D4E0004A680720032A2FD90C1C1B4899B202AAAC
:10D4F000FCF71EFE002827D101A802A904226423FC
:10D50000FCF7B0FE002804D1019B013301D0134E7B
:10D5100000E0134E211D02A804226423B047002816
:10D5200012D102A8A16810226823FCF761FE00282E
:10D530000AD1AB78A1680B4A9B00995004E00A48D5
:10D5400002E00A4800E00A4804B070BD542A0020F6
:10D55000FC2A0020642A00200C2B0020F1A10100ED
:10D560007DA10100442A00200E80000008800000F8
:10D57000108000001FB5244B1B78002B3DD00028E5
:10D5800039D0002937D00378002B36D11F4B1B68C8
:10D59000002B32D08378022B31D81C225A431C4CEA
:10D5A000A218927EFF2A2AD08C681A4A9B00002C6F
:10D5B00002D1D3588B6000E0D4500C1C02AA8178B1
:10D5C0001548FCF7B5FD00281CD101A802A90422CA
:10D5D0006423FCF747FE002813D1019B013310D0D0
:10D5E000A06802A910226823FCF73CFE002809D19C
:10D5F000019B636006E0094804E0094802E009482D
:10D6000000E0094804B010BD542A0020FC2A002084
:10D61000642A0020442A00200C2B00200E800000E9
:10D620000880000010800000408000001FB51E4BE5
:10D63000041C1B78002B31D000282DD00378002B40
:10D640002CD11A4B1B68002B28D08178022927D8AF
:10D650001C204843164B1818837EFF2B20D089B21C
:10D66000144802AAFCF764FD00281AD1642301A81B
:10D6700002A90422FCF7F6FD019B013311D002A898
:10D680000D4904226423FCF7B3FD002809D1A378D7
:10D690000A4A9B00985004E0094802E0094800E06B
:10D6A000094804B010BDC046542A0020FC2A0020BE
:10D6B000642A00200C2B0020741C0200442A002045
:10D6C0000E8000000880000010800000002806D0B6
:10D6D000FF23037043708370C370002000E0014893
:10D6E0007047C0460E80000010B5194A031C12781E
:10D6F000002A29D0002825D0002923D00478002C26
:10D7000022D1144A1268002A1ED09A78081CFF2AD7
:10D710000AD15978FF2919D00C2359430E4B5918B7
:10D720008B7A9B0712D508E01C21022451430B4B36
:10D7300059188B7E1C4009D11031072203F02CFFB1
:10D74000201C04E0064802E0064800E0064810BD40
:10D75000542A0020FC2A0020562A0020642A002097
:10D760000E800000088000000580000013B5041C36
:10D7700081786A460B48FCF7DBFC002810D11C239B
:10D780006078094A5843694610181A1CFCF76AFD6C
:10D79000064B074A9B7A68469B009B58211C98477A
:10D7A00013BDC0460C2B0020B82A0020FC2A002004
:10D7B000541C0200F0B5FF24C34B8FB01B780394B8
:10D7C000002B00D1D4E1C14B1A680093002A00D18C
:10D7D000CEE105AF031D7B602A2300223B81038835
:10D7E00004AD6C70AC70EC70061C2A70B84C102B39
:10D7F0000AD0A27A8188900766D5B648814208D0BF
:10D800002089884260D104E00121A37A0B4205D12E
:10D81000AEE1E17AA9700021697055E00223A3729C
:10D8200011236A703B708388871D23810722201C87
:10D83000391C03F0B1FE0123327D134006D0A64B04
:10D8400052089B5CFF2B32D0039330E01C1CA34E8C
:10D850001C20604310303018391C072203F072FE80
:10D86000002801D1039422E00134032CF0D102E01E
:10D87000F379034240D10024009B05AE1B68281CAD
:10D88000311C221C98473378122B00D070E190484D
:10D89000837A012B00D16BE10123837201235B4268
:10D8A0000381C3720021072203F0B8FE60E1082063
:10D8B000874A039B917ADBB20143D3729172281C91
:10D8C000AB70FFF753FFD6E7172B5FD1012704207A
:10D8D0001424009B00995B7A8243BB434B727C4BC0
:10D8E00005A90C709A72B479191C002CC0D0D87A92
:10D8F000FFF716FCB479BFE7AC78FF2CBBD0082348
:10D900001A43F37A8A729B0706D51C236343734A32
:10D91000D3189A7EBA439A76CB7AFF2BABD01C26CB
:10D9200066436E4F0B78BE19022B09D0301C0722BC
:10D93000103003F031FE0222B37E9343B37606E04B
:10D940000121674B5B8A3383B37E8B43B37600261A
:10D950000197A6420FD0019B9B7EDB070BD41C20B6
:10D96000604301993818102203F0ECFD002802D121
:10D97000301CFFF7D5FB019B01361C330193032EAE
:10D98000E7D1281C0121FFF7ABF974E7172B00D969
:10D99000B7E0132B5BD113233B7004231A43E37AC4
:10D9A000A272FF2B2CD14D4B9B7EFF2B0BD04B4BF0
:10D9B00036331B78FF2B08D0484B022752331B7895
:10D9C000FF2B2BD102E0002700E001272378FE2265
:10D9D000022B09D01C207843404B07221818103026
:10D9E000211C03F0D9FDFD221C237B433B49CB18AE
:10D9F0009A7603AB1F70039BDBB2AB70E3720BE054
:10DA0000162338482022083000213B7003F006FE20
:10DA10004022A37A1343A372002400E0324C002179
:10DA20002B4B0B91DA7A1C2353432C4A0D91D318BC
:10DA30000C932B4B09910893009B0A911A1DB088F7
:10DA400008ABFFF734F9002800D115E790E0142B5C
:10DA500029D1E37A214FFF2B1AD1F389398B9942CF
:10DA600009D0B98E994208D0391C503109889942A1
:10DA70000ED1022302E0002300E0012308210393DA
:10DA80000A43DBB2E372A272281CAB70FFF76EFE92
:10DA9000E37A0021FF2B00D01149B0883A1C002303
:10DAA000FFF707F964E0112B62D10223111C99439F
:10DAB000A17212071AD54BB2002B1EDA281C0021C6
:10DAC000FFF70EF919E0C046542A0020FC2A002076
:10DAD000562A0020FFFF0000502A0020642A002060
:10DAE000B82A0020D42A002043800000A878FF280C
:10DAF00003D0FFF7EDFAFF23AB701023A3721223BC
:10DB000002E01C2B02D113233B70B4E6522B07D149
:10DB1000009B184A9B7A281C9B009B58984727E03B
:10DB2000182B25D1B379112B14D1130712D5124814
:10DB300020220830002103F071FD162360223B7083
:10DB4000A37A13430222A372009B5B7A1343009AC9
:10DB5000537290E680235B421A4315233B70009B6F
:10DB6000A2729B7A034A9B009B58281C984782E626
:10DB70000FB0F0BD641C0200D42A0020A1230321B1
:10DB80000B4ADB00D150802300210A4A9B00D15070
:10DB9000094B5961012111615969064A0029FBD0DD
:10DBA000002305494B6153601360044A138070479A
:10DBB00000F0014000100040FC1000401E2B00202F
:10DBC000A8220021124BD20030B59950A722114C47
:10DBD000D2009C50104C114A03259C50A124104A9D
:10DBE000E4001268520002321A510E4A0E4C9C5048
:10DBF00080240E4AA40051601D51884203D0116157
:10DC000001225A6003E00A4A11680A4A995030BD5D
:10DC1000001000405B060000555555003C05000013
:10DC2000202B002004050000252B0020FC100040C4
:10DC30001C2000200C050000002238B5434B0121B8
:10DC40005A608022D20511605A68002AFCD0002256
:10DC500001213F4B3F481B6880245960D9601A500E
:10DC6000181CFC3042648264C2640265C1206402F4
:10DC700080001C50802080001950A2200424C00085
:10DC80001C50A820344CC0001C508224334864002F
:10DC90001C501960324B1A60324B1B681B0716D49C
:10DCA000314B324A1968324B9950324A1168E52299
:10DCB000D2009950304A1168304A9950304A116860
:10DCC000E622D20099502F4A11682F4A99502F4BC3
:10DCD00004201D68FC232C1C9C4335D12B1C2833AD
:10DCE000DBB22C2B30D8FFF749FF214B284A032108
:10DCF0009D50A222FF20D2009950264A9958814374
:10DD0000712099509958014399502349234A04207E
:10DD10009950A6210122C9005A502149FF305C5078
:10DD2000204958508420204940005850A3211F48C2
:10DD3000C90058501021201C1D4B1C701D4B1A701F
:10DD40001D4A13690B43136138BDC046FC000040F7
:10DD500014200020040500007102000044050000AA
:10DD60004C2B0020AC000010EC0000102407000039
:10DD700000100040F0000010F40000102C0700001C
:10DD8000F8000010FC000010340700001C200020E8
:10DD90000C05000024050000002941761C05000048
:10DDA0002C050000340500001405000025000300C8
:10DDB000242B00201C2B002000ED00E0102138B5A2
:10DDC0002F4A304D1369304C0B4313612F4A304BAF
:10DDD0001169002936D000211161C02202202D498D
:10DDE000520088502A78042A2CD101225A608022BD
:10DDF000D2009B58012B20D10F2321786278194043
:10DE000081421AD8252A18D800290AD12018224977
:10DE100003F098FB002810D1204A138801331380A7
:10DE20000BE0012900D055230021C8B29042F3D263
:10DE30000131601840789842F7D0201C0021272239
:10DE400003F0ECFB164B1B68FC335A6C002A02D023
:10DE500000225A64BAE7996C0029B7D09A64114B32
:10DE6000012219781F230B409A40131CC022094934
:10DE700052008B500C4B1A68501C186038BDC046BD
:10DE800000ED00E01C2B0020252B0020FC100040A2
:10DE90000010004000E100E0781C02001E2B002072
:10DEA00014200020182000204C2B00200021044BBF
:10DEB0001A781970034B1B880360101C7047C0460A
:10DEC000242B0020142B0020084A031C1278002069
:10DED000012A09D81A1C2832D2B22C2A04D89A074F
:10DEE00002D10120024A13607047C0461C2B00205B
:10DEF0001C2000200E4B1A780023012A16D89842C5
:10DF000004D10C4A0C4B1A6008220CE0012804D101
:10DF10000A4A094B1A60092205E0022806D1084A7C
:10DF2000054B1A600A22074B1A700123181C704710
:10DF30001C2B002000800040142000200090004096
:10DF400000A0004018200020F7B56D46041CD0B298
:10DF500001902D7960480127057000255F48036016
:10DF60005F4801605F4807705F4805805F48007840
:10DF7000844666460520AE4200D1ABE0AC420DD1EE
:10DF8000A8235B4ADB00D450A1225A4BD2009F50F9
:10DF9000A222D2009C50584A9C501BE0032C1ED158
:10DFA000012E04D10123504A0220138092E0534BEA
:10DFB000534A1B8813434C4A1380A8234C4ADB0066
:10DFC000D550A1224B4BD2009F50A222D2009D508F
:10DFD000494A9D50FFF7D2FD444B1F7079E06046DF
:10DFE000012EDFD1272902D93F4B1E8072E0434822
:10DFF0000580012C09D1291C2722424803F00EFB81
:10E00000201CFFF7DDFD042361E0281C022C61D1F8
:10E010000198252803D9344B03201E805AE00F2491
:10E02000181C384D20402870684600796870281CFC
:10E03000012B0BD0002B04D0022B0AD001330DD0C2
:10E040002EE03149023003F0A7FA2EE0A81C211C73
:10E0500001E05521023003F0E1FA26E00020032A16
:10E0600038D8101C03F05AFA020212180020FFF7E9
:10E07000A7FDA82103221E4BC90080205A50012170
:10E08000800019501960194B1A7022E0081CFFF724
:10E090001BFF002807D01CE0081CFFF72BFFF8E748
:10E0A0000123114A1380042014E00020FFF788FDAB
:10E0B000A221164BC9001A680E4B4132FF325A504A
:10E0C0000B490D4A99500121114A99500223074AE0
:10E0D00013700020FEBDC0461D2B0020182B002011
:10E0E000202B0020242B0020142B00201C2B002090
:10E0F0000010004000F00140140500001E2B00201D
:10E100000080FFFF252B0020781C02001420002037
:10E110000405000010B51A490B78012B19D1194BD1
:10E120001B681B0715D1184BE0241A68F023101C3C
:10E13000184022420BD1154A12681A4209D1144ADA
:10E14000144B1A608022144B12021A6001E030282E
:10E15000F1D00978012912D10A4B1B681B070ED197
:10E16000F022094B1B681340402B08D1074B1B685A
:10E17000134204D1C1238022DB00D205D15010BD4F
:10E18000E00F00F0E40F00F0E80F00F0EC0F00F0FB
:10E19000DFFF07C004050040186C00402EDF704709
:10E1A00051DF704710DF704711DF704761DF704744
:10E1B00008B5081C111CFCF705FC08BDF0B5274B81
:10E1C00085B01B78002B47D0254D264E2B68346830
:10E1D0005A425341DBB2009363425C41E4B2009B7C
:10E1E000002B37D103A8FFF7DBFF05280AD0002852
:10E1F00004D000210A1CFCF7C1F905E003982B6844
:10E20000984701E001230093002C1FD1164B03A96E
:10E210001B8801240B80154B1B68181C0193FFF70A
:10E22000C5FF071E052F0BD0002805D000210A1CB2
:10E23000FCF7A4F9002403E00198336898473C1CDC
:10E24000009B002BCED0002CC9D005E0009B002BFA
:10E2500002D1C7E7002CD9D005B0F0BD502B00206B
:10E26000582B00205C2B0020522B0020542B002028
:10E2700038B5041C0720002913D08D0711D1094897
:10E2800001600949201C0A80084A09491360FFF708
:10E2900089FF002805D10122064B16201A70FFF7CE
:10E2A0007DFF38BD542B0020522B0020602B002016
:10E2B000B1E10100502B002008B5FFF775FF031CEA
:10E2C0005A1E9341014ADBB2137008BD502B002047
:10E2D0000E23002802D0024B18600023181C704740
:10E2E0005C2B00200E23002802D0024B1860002374
:10E2F000181C7047582B002008B5074B1B68002BD3
:10E3000007D09847002806D000210A1CFCF736F9F0
:10E3100001E0FFF753FF08BD602B002008B500297E
:10E3200004D00020011C021CFCF728F9FFF746FF6F
:10E3300008BD0000002008B5011C024AFAF7EAFEF9
:10E3400008BDC0461DE30100A023EF220021DB052C
:10E35000D20070B5012099501D1C20220426094CC2
:10E36000011C9140214204D0111CC131FF318900B0
:10E370004E51013AF4D2A321034AC9005A5003492D
:10E380005A5070BD5300C022AC9F05080C05000018
:10E39000A023A321134ADB05C90070B55A500028F9
:10E3A00004D0A121C9005A50022001E00E495A5060
:10E3B0000422A0262023012400040C4D0243F6056C
:10E3C000211C9940294204D0191CC131FF31890018
:10E3D0008A51013BF4D2EF23A022DB00D205D050BA
:10E3E00070BDC046AC9F05080C0500005300C0225C
:10E3F000A223A0220120D205DB00D3589B0F984313
:10E400007047000030B5A024202301210B480C4D9B
:10E41000E4050A1C9A40024204D01A1CC132FF32A1
:10E4200092001551013BF4D2A023A321054ADB053C
:10E43000C9005A50A121C9005A5030BD5300C02212
:10E4400004000200AC9F05080022F0B587B00A70F6
:10E450000D230292A02203900193D205A325019BD4
:10E460003A48ED005C1E019469D3394B394CD050C9
:10E4700010515051D050019C374BE35C0124261CB5
:10E480009E405651A125ED005651C046A223DB0007
:10E49000D5582E02F60FA640AF0927403E432F1C49
:10E4A000AB07DB0F9B001E43EB06DB0FDB001E43BD
:10E4B0002740AB003F01DB0F3E435B0133436E025D
:10E4C000F60FB6011E43AB01DB0FDB01019D3343A9
:10E4D000224EAD00AB51002BC0D0019D0026EF00B5
:10E4E0001F4D0594ED1904950825013D17D3059F8F
:10E4F000AF401F42F9D00F78052F0ED8049C675DFE
:10E50000BC466446039F3C703C1C013403940C7869
:10E51000A4460124A44464460C700136E5E7012EAC
:10E5200009D9029C1C4206D0A323A022DB00D205FD
:10E53000D050002007E00298184302908EE7A023F5
:10E54000DB055851012007B0F0BDC046AC9F05085F
:10E550001C0500000C050000081D0200642B0020B3
:10E56000A01C0200F0B50023042A1AD108250226B7
:10E570000127041D0178132901D13B430AE0042936
:10E5800001D1334306E00C2901D1134302E01529E0
:10E5900000D12B430130A042ECD10F3B5A425341F2
:10E5A000DBB2181CF0BD2EDF704732DF704733DF5F
:10E5B000704712DF7047000070B52D4C6368002B68
:10E5C00003D1A368002B0FD10AE00025294E656016
:10E5D000337A9D42F5DAAB009B5998470135F7E74E
:10E5E000E368002B11D10CE00025214B214E9D60EA
:10E5F000337D9D42F4DAAB00F318DB6898470135B0
:10E60000F6E72369002B18D10DE00025184B194EB1
:10E61000DD60731CDB7F9D42F3DAAB00F3189B696E
:10E6200098470135F5E7BE23134A5B00D15800290E
:10E630001DD000240F4DD4500EE000240C4B0D4D86
:10E640001C612B1C2C331B789C42ECDAA300EB18CA
:10E650005B6A98470134F4E72B1C38331B789C42E3
:10E6600005DAA300EB181B6B98470134F4E770BD83
:10E67000FC600040982B00200060004037B500206F
:10E680006B46164CDD1DD8712378834224D1281C9B
:10E69000FFF78FFF00281FD12B78012B0AD1032110
:10E6A0000620FFF784FF0620FFF77FFF0620FFF715
:10E6B0007AFF0EE0C1210A4A89005058094B0340F5
:10E6C000C020000403435350C0214023490053504D
:10E6D00013600123002023703EBDC046D42B0020D0
:10E6E00000E100E0FFFF00FF30B50723042838D821
:10E6F0000C2242431C4D0423AA18147A012C30D852
:10E70000032343431B199B00013414725951C12444
:10E710004A1E91410138C9B2144A0023A4000328BB
:10E7200004D8251C02F0FAFE060A101410484360B3
:10E73000115116E00E484900836002E00C48890040
:10E74000C360515100230CE00948C9000361F8E798
:10E75000002901D0802109061151BE210023490062
:10E760005350181C30BDC046982B0020006000405C
:10E77000FC6000408122F8B52648274B5200C25069
:10E78000A0230124DB00C4508022A023A121002566
:10E79000C900DB0592035A5020494D6004604C6863
:10E7A0001C48002CFBD01E4901255A50A123DB0038
:10E7B000C3581C4C45605C431B4802F07FFD201C85
:10E7C00002F0A4FD194802F079FD194B64209C4227
:10E7D0001ED82B1C174A990089588C4214D9164808
:10E7E0005D1EC65C475D601AFA24AD00AB58A400FC
:10E7F000591A604302F06EFEBF1B7843211C02F0E1
:10E8000069FE3018C0B203E00133072BE3D10020CA
:10E81000F8BDC0460070004004050000FC700040D8
:10E820000C050000D5100000181D02002B1D020071
:10E830000B7941003C1D0200341D0200A023802200
:10E84000A321DB059203C9005A50024900205A5007
:10E850007047C0460C05000074DF704776DF7047D4
:10E8600078DF70477ADF70477CDF70477EDF704764
:10E8700080DF704760DF70472FDF7047002330B5BF
:10E8800087B001A80193FBF76DFD041E1BD1019D0C
:10E890000123002D07D00D4A137010230C4A116874
:10E8A0000B4313600FE002A98860C86009480B7031
:10E8B000FEF7A0FD0823021C041C9A4303D0291C68
:10E8C0002A1CFBF75BFE201C07B030BDB62E0020D3
:10E8D000F42E0020B82E00201FB50368041C187801
:10E8E000072850D802F01AFE54540454283D3F43E0
:10E8F000284A13780133DBB21370274A12789A4200
:10E9000046D8264B01A81B689A8DC2801A8D42807A
:10E91000DA8C02805B8D8380FCF7D6FF112805D04E
:10E92000002803D000210A1CFBF728FEFFF7A6FFF2
:10E93000002100282CD028E0A268002A03D1101C56
:10E94000111CFBF71BFE032301A80370237903713D
:10E9500063794371A3798371E379C371A368836099
:10E960000CE0012200E000220D4B1A7010E004239D
:10E9700001A8037023790371A3794371094B0C211A
:10E980001B68984704E00020011C0A1CFBF7F6FDF9
:10E990001FBDC046F82E0020002F0020F02E0020C2
:10E9A000582E0020242C0020F0B589B0061CFBF75F
:10E9B0003FFA022E7AD1404B1A780193002A75D083
:10E9C000002403A80394FBF7CDFCA04203D0211C34
:10E9D000221CFBF7D3FD039D002D67D10122374C8C
:10E9E0002368134218D093432360354B1868FBF714
:10E9F00037F8002803D0291C2A1CFBF7BFFD00258F
:10EA000004A80C212F4A0570FAF784FBA84203D012
:10EA1000291C2A1CFBF7B2FD0422236813420ED0E6
:10EA2000934323600D2304A80C21264A0370FAF7B0
:10EA300071FB002803D000210A1CFBF79FFD08276B
:10EA400023681F400AD008221F489343236000F028
:10EA50007DFE002825D000210A1C20E020221D1C5C
:10EA6000154009D093431848236000F0C3FE0028E6
:10EA700017D0391C3A1C12E01022134211D09343D4
:10EA80002360012304A910480B708D60CD60FEF750
:10EA9000B1FC0822031C934303D0291C2A1CFBF75A
:10EAA0006DFD2368002B01D1019A1370301C01F019
:10EAB000C1FA09B0F0BDC046B62E0020F42E0020E9
:10EAC0002C2C0020B1ED0100B82E002037B5041C1D
:10EAD0000D1C0B78002A06D0322B04D1FFF7CEFE96
:10EAE00000280DD008E0142B03D1842A08D0812AF5
:10EAF00006D0002A04D0101C00210A1CFBF73EFDA2
:10EB00002B78152B37D004D8112B23D0142B2CD0D5
:10EB10005EE0212B29D0222B5AD16846FBF722FC3C
:10EB2000002803D000210A1CFBF728FD009C002CC4
:10EB300007D1284800F00AFE002849D0211C221CD9
:10EB400044E00122244B1A700823244A11680B4325
:10EB500013603DE0A378FF2B3AD08021204B49027F
:10EB600018680022FAF726FF32E0211C0422194817
:10EB700002F012FD2CE001221A4B1A701A4B1C787D
:10EB8000002C15D16946194B68461B689A8DCA80BE
:10EB90001A8D4A80DA8C0A805B8D8B80FCF794FE9C
:10EBA000112805D0002803D0211C221CFBF7E6FC0D
:10EBB0000122A0210E4B49021A700E4B0022186848
:10EBC000FAF7F8FE002803D000210A1CFBF7D6FC58
:10EBD00000203EBDB82E0020B62E0020F42E0020CE
:10EBE000AC2E0020EC2E0020B72E0020F02E0020AE
:10EBF000282C00202C2C002070B5027F041C07203C
:10EC0000042A1DD81C230F49024095000A780226C9
:10EC10009A432A4313400C3B5D1EAB410125AB4098
:10EC2000B2431A4310232A430A7048708B70637FE3
:10EC300000201D40D3B220226D0193431D430D706F
:10EC400070BDC046B12E00201FB50B78002B05D13A
:10EC50000C21034B01A801701B68984705B000BD4B
:10EC6000242C002008B5072805D0002803D0002157
:10EC70000A1CFBF783FC08BD10B5084B1C78002C60
:10EC80000AD1074B07491888FFF7F0FD002803D089
:10EC9000211C221CFBF772FC10BDC046EC2E00208C
:10ECA000362C0020B12E002008B5002803D000210A
:10ECB0000A1CFBF763FC08BD13B51D4B1A78002A2C
:10ECC00029D01C4A1278002A25D01B4A11881B4AD9
:10ECD000914220D0002401A81C70FBF743FBA04206
:10ECE00003D0211C221CFBF749FC019C002C09D1FC
:10ECF000134800F07FFD002819D0211C221CFBF7CF
:10ED00003DFC14E001220F4B1A7020230E4A1168BB
:10ED10000B4313600BE00B4B1B78002B07D0BFF3AA
:10ED20004F8F0A4A0A4BDA60BFF34F8FFEE713BDDD
:10ED3000282C0020EC2E0020362C0020FFFF0000A5
:10ED4000B82E0020B62E0020F42E00200400FA0574
:10ED500000ED00E007B5124B122012494822FFF7E0
:10ED600087FA002803D000210A1CFBF707FC0822C1
:10ED70006846002102F052FC6B4601221B7868466F
:10ED800013436A461370FFF775FD002807D1064844
:10ED9000FFF79EFA002802D10448FFF7A3FA0EBD40
:10EDA00035E30100642E00208DF40100A9E9010083
:10EDB00038B5051C16200C1CFFF75EFD002803D09B
:10EDC00000210A1CFBF7DAFBFFF776FA002803D0D4
:10EDD00000210A1CFBF7D2FB0C2C04D1024B281C8F
:10EDE0001B68211C984738BD242C0020F0B50B1C53
:10EDF0008DB00721002800D1D4E0041CC0206B4D49
:10EE00004002191C38220193286002F09BFB002865
:10EE10001CD08023664A5B051E695169013105D00B
:10EE20005069196989B202F055FB00E05869464300
:10EE3000604B9E4204D80020011C021CFBF79EFB85
:10EE4000C020019940020E2202F0F0F95A4B5B48B3
:10EE50001C6000242B68211C5A6B594B1A6001223C
:10EE6000584B52421C70584B1C70584B1C70584BDE
:10EE70001A80584B48221C7002F0D0FB564F211CC0
:10EE80000522381C02F0CAFB211C1822534802F04C
:10EE9000C5FB211C0222524802F0C0FB514B524ECE
:10EEA0001C70524B211C5248524A1C703460FAF7B5
:10EEB0005BFD011EA14275D12B6806A8DA8D028286
:10EEC0001A1C3032127882741A1C31321278C274D1
:10EED0001B7F0375484B83608023DB00C360474B77
:10EEE0000693474B436001F02BF9011EA14259D113
:10EEF000FFF730FF011EA14254D1FBF733F8011E8A
:10EF0000A1424FD12868FFF777FE011EA14249D1E7
:10EF1000019B3C480433DD7FFEF7D8FB011EA14274
:10EF200033D102AB181C1D70FEF710F9011EA1426F
:10EF30002BD1092002ABC018052202F06FFB3B78F1
:10EF40000120191C03AD6A79014082435C0804402A
:10EF50000A43022184408A4322431C211C24194075
:10EF6000A2430A4320215B0903405B018A431A4301
:10EF70006A717B78291CAB71BB782871EB71224BCD
:10EF800022480393FEF758F9011C00290AD10123F6
:10EF9000144A1F481370326813431E4A3360FAF74D
:10EFA000E3FC011C081C0DB0F0BDC046F02E002093
:10EFB000001000100D800100242C0020D82B002010
:10EFC0005C2E0020EC2E0020B72E0020582E0020B2
:10EFD000362C0020002F0020B12E0020042F00200E
:10EFE000602E0020B62E0020F42E0020202C0020C1
:10EFF000AC2E002079EC010000810100D9E801006D
:10F0000065EC0100B82E0020CDEA0100352C00206F
:10F010002C2C0020B9EC010008B5034B021C012187
:10F020001888FFF725FC08BD362C0020F0B51F1C02
:10F03000184B85B01B78051C0824002B27D00B1C0F
:10F040001549101C09782A1C002919D00F26802187
:10F050006E443170114D1249009001970F68281CC1
:10F06000311CB8473378201CDB0702D5281C01F07F
:10F0700063FB33789B0706D5281C01F073FB02E085
:10F08000391C01F04BFB0022041C064B1A70201C9B
:10F0900005B0F0BDEC2E0020582E0020382C0020AA
:10F0A0005C2E0020B02E002008B5011C0348FCF7A0
:10F0B00079FA0022024B1A7008BDC046042F0020C6
:10F0C000B02E0020F0B501269E4B9FB00190DE6768
:10F0D00001F066FB02300424052800D92EE1FFF779
:10F0E00039FE041E00D029E110232422964F1E432E
:10F0F00002AB9B183D681E702C68201C02F0DAFAE7
:10F10000211C82B20BA8FFF7AFFB041E0ED1A88C06
:10F11000FFF7A6FB041E09D1291C082226310EA8E0
:10F1200002F03AFA0EA8FFF79DFB041C002C00D059
:10F1300004E124213E6802AAB37D52181370B38AF9
:10F1400002AAD384338B0EAD1385738B211C538598
:10F15000281C402202F062FA7168002902D0281CA3
:10F16000FDF79CFDB168002902D014A8FDF796FDBB
:10F17000F168002902D016A8FDF790FD3169002939
:10F1800002D012A8FDF78AFD11220BABAB631DABB9
:10F190001A706D23002202A95B18281C1A70FCF754
:10F1A00041FE041E00D0C9E005AE211C301C0C221B
:10F1B00002F034FA654B664873600123311CB46079
:10F1C0003380FCF7C3FB002803D0211C221CFBF773
:10F1D000D5F90EAE00211422301C02F01FFA0124D2
:10F1E00000235C4A34710E935378591E8B415B4265
:10F1F0001340AB60FFF7BEFA10231A1C22436A7358
:10F200001A1C2243AA7300221C432873291C52484B
:10F210002C74EA73FCF7FEF8041E00D08EE04F4E0B
:10F220004F4B32781968737838681B021343B278F1
:10F230001E3012041A43F3781B061343494A00F0A8
:10F240005DFC002879D13E68211C1C22281C02F09C
:10F25000E5F9311C082226310BA802F09DF90BAB11
:10F260002B6080231B026B60F0231B03AB603E4BC3
:10F270000326AB610123281C5B422C746C612E7346
:10F28000EB81FCF789FA041E58D13868FFF7B4FC0B
:10F29000002852D101F0C8F800284ED1019B002B64
:10F2A0004CD0201C00F052FC341C002846D000F04A
:10F2B000EDFC041E052C41D12C4E02ABDD1C307838
:10F2C00003A92A1C00F056FB002836D12B78002B0E
:10F2D00003D1301CFEF762F822E004AD281CFEF7D3
:10F2E000F5F9337800262B7000230C270893FF21B3
:10F2F0000BAB3A1C0EA80A93AE70099702F08EF978
:10F30000281C08A9FEF736F9041E12D10BA80EA975
:10F310003A1C02F017F900280BD1281CFEF720F840
:10F320000123134A041C1370124A11680B43136023
:10F3300004E00136032ED7D100E0041C201C1FB0CE
:10F34000F0BDC04604E100E0F02E002049EC0100D1
:10F35000BC2E0020602E0020042F0020B82E00209C
:10F36000242C0020EC2E0020A9EC0100352C0020DC
:10F37000B62E0020F42E002008B500F06BFF08BD6B
:10F3800073B506AC2678012903D1054D2C780134DC
:10F390002C70079C0096019400F0CCFF76BDC0460F
:10F3A000002F00201FB50C4C0C4B2088984208D031
:10F3B0001321FFF753FA00280CD101235B4223806D
:10F3C00008E0022301A80370054B0C211A68F9F725
:10F3D000A1FE002004B010BD362C0020FFFF00006D
:10F3E000242C002030B585B06846FAF7BBFF041C1A
:10F3F000011E3CD1009C002C09D001221D4B0C1C8D
:10F400001A7004231C4A1068034313602FE01B4D3D
:10F410001B4B288898420BD01321FFF71FFA0028B6
:10F4200024D1012301225B422B80164B1A701EE06F
:10F43000FCF7EAF9002819D1FFF70EFA6846FAF747
:10F4400091FF002812D1009B002B08D00122094B0C
:10F450001A700423084A11680B43136007E00D2358
:10F4600001A80C21084A0370F9F754FE041C201C63
:10F4700005B030BDB62E0020F42E0020362C002022
:10F48000FFFF0000202C0020B1ED0100F0B5038843
:10F4900085B0041C012B3FD15D4A5E4C137023687C
:10F4A000002B00D1B1E05C4E5C4F2368EF211A1CA9
:10F4B0000025FC329268307891426D4113359A18DC
:10F4C00039782B1C01F02AF9002800D09DE0236830
:10F4D000132D1CD1FF335872514B524D1A68012322
:10F4E00013702A1C2060FF32517A2A1C002905D192
:10F4F00085218900695C002905D0181C86235B00E2
:10F500005843101820602368002BCED17DE0FC33D7
:10F510009A6814329A60C8E7FEF74CF9201CFCF791
:10F520007BF9201C01F0E4F8201C00F057FD3E4858
:10F53000211CFBF746FF3D48211CFCF75DFB2088A2
:10F540001038092861D801F0E9FF0F1A053B606007
:10F550003F596034052301A80370E38883806389E1
:10F56000C380A38903814CE0A288314B01A81A8093
:10F570000023304A1370304A1370012340E0012207
:10F5800000242B4B52421A802C4B1C702C4B1B78A6
:10F59000A34207D0FFF726FFA04203D0211C221C64
:10F5A000FAF7ECFF00F068FD00282ED101A8022335
:10F5B00026E000F061FD002827D101A806231FE006
:10F5C00001221E4B1A7020E0A379012B04D0022BDC
:10F5D00009D101A80A2301E0092301A80370194BEE
:10F5E0000C211B689847184B1868FAF739FA00285D
:10F5F0000BD000210A1CFAF7C1FF06E00B2301A87B
:10F600000370104B0C211B68984705B0F0BDC04635
:10F61000B02E0020302C0020342C00201C2F002085
:10F62000FC2E0020402C0020042F0020BC2E0020A7
:10F63000362C0020EC2E0020F82E0020B72E0020C3
:10F64000202C0020242C0020AC2E002008B5054BD7
:10F6500001201A88044B9A4202D0FFF7A3FE002033
:10F6600008BDC046362C0020FFFF0000014B187873
:10F670007047C046B02E002071DF7047F0B5041C03
:10F680008BB003AE301C0191FEF720F823780024E4
:10F6900033700C23251C07AF05930697301C04A973
:10F6A000B470FDF767FF002805D13B68AB4202D973
:10F6B0005A1C00D01D1C0134E4B2032CEED10020F2
:10F6C000019B01351D600BB0F0BD0000F0B5041CBE
:10F6D00087B005AE301C02910392FDF7F7FF237847
:10F6E000184D337063780024174F737001940C2306
:10F6F000AF606B60301C291CB470FDF73BFF002825
:10F7000013D13B68019A9A4200D20193029A934224
:10F710000BD9013B3B60301C291CFDF7C3FE0028C0
:10F7200003D000210A1CFAF729FF0134E4B20C359A
:10F730000C37032CDBD10020039B019A1A6007B021
:10F74000F0BDC046842F0020202F00200C23F0B5F0
:10F750008578244F5D4379194B60234B85B05B1945
:10F760008B60041CFDF706FF0197061E1E4F09D192
:10F77000E959201C03AAFFF7A9FF00280CD0311C6F
:10F78000321C07E0201C03A9FFF778FF002803D0F4
:10F7900000210A1CFAF7F2FE0C22A078019B5043CC
:10F7A0001B183818114F124D386098605A60043099
:10F7B000039E2B60FFF760FF002803D000210A1C86
:10F7C000FAF7DCFE3B6829681E60201CFDF76AFE24
:10F7D000002803D000210A1CFAF7D0FE002005B053
:10F7E000F0BDC046BC2F0020542F0020EC2F00207D
:10F7F000B82F00200C23F0B585782B4F5D43791985
:10F800004B602A4B87B05B198B60041CFDF7B2FE7E
:10F810000197061E254F43D1ED59201C291C03AA30
:10F82000FFF754FF002803D0311C321CFAF7A6FE64
:10F83000039B00939D4233D00C21A378019A4B4344
:10F840001B4DD218FF181B4E5160976004A82A6008
:10F850003760FFF711FF002803D000210A1CFAF7D8
:10F860008DFE201C2968FDF785FE002803D00021AD
:10F870000A1CFAF783FE336804A9181D072201F059
:10F8800061FE071E0CD13368009A29681A60201C9B
:10F89000FDF708FE002803D0391C3A1CFAF76EFE6B
:10F8A000002007B0F0BDC046BC2F0020542F002020
:10F8B000502F0020B42F0020F0B5041C002687B084
:10F8C00004A8039301910292FDF700FF04AB274DBA
:10F8D000274F1C706A46F3B20093127804AB9A70FB
:10F8E0000C23AF606B6004A8291CFDF743FE041EC7
:10F8F00034D13B68019A013B93420ED10C235E4305
:10F900001B49072289190431029801F045FE6A4615
:10F91000039B1278201C1A7026E002331ED104A823
:10F9200005A9FFF7ABFE002803D0211C221CFAF723
:10F9300025FE381C059B08C0FFF79EFE002803D05B
:10F9400000210A1CFAF71AFE04A8291CFDF7AAFDDB
:10F95000002803D000210A1CFAF710FE01360C35EE
:10F960000C37032EB6D1052007B0F0BDBC2F002008
:10F97000542F0020F0B5051C85B003AC201C0F1CD3
:10F980000192FDF7A3FE25700024251C104EE3B262
:10F9900000936B461B7803A883700C23736063434A
:10F9A0000C4A311CD318B360FDF7E4FD002805D1E3
:10F9B0006B461B7801353B70EDB2013701340C36D4
:10F9C000032CE4D10020019B1D7005B0F0BDC046A2
:10F9D000BC2F0020542F0020F0B5041C85B003AECE
:10F9E000301C00910192FDF771FE34700024154D1A
:10F9F000154F0C23AF606B60301C291CB470FDF7F1
:10FA0000B9FD002814D13B68009A013B934205D10F
:10FA1000019B301C1C70FDF709FE07E0009A934221
:10FA200006D93B60301C291CFDF73CFD002806D19F
:10FA30000134E4B20C350C37032CDAD1002005B0C8
:10FA4000F0BDC046BC2F0020542F002070DF70474F
:10FA500071DF704773DF70470C23F0B589B001ACDC
:10FA6000051C0393201C05AB0E1C0493FDF72EFE12
:10FA7000002803D000210A1CFAF780FD257000271A
:10FA80000024002501A802A98770FDF773FD002856
:10FA900015D105AB9A79D9791202090458790A432C
:10FAA000197A024309060A43597A9B7A1B020B43CF
:10FAB000AB4202D803D1A24201D9141C1D1C01374C
:10FAC000FFB2032FDED1231C08202B4313D00122C9
:10FAD0000023A4185D410123402200203370230A33
:10FAE000B370230CF370230E337152422B0A13436D
:10FAF00074707571B37109B0F0BD000013B5019356
:10FB00000723002815D0002913D0002A11D0002483
:10FB1000094B18600079094B1870094B09481960A6
:10FB2000094B04701A600130211C052201F076FD9A
:10FB3000231C181C16BDC046F42F0020FE2F0020E9
:10FB4000F02F0020F82F002000300020F7B54B4B9D
:10FB5000051C18786B46DE1C01A9321CFFF70AFF52
:10FB60000124071E00D087E0454B5C781878002CF4
:10FB700036D004282DD801F0D1FC037E1B231B00B6
:10FB8000404A1268D478002C10D0317800293CD13A
:10FB90000CE0002D31D02A88112A2ED13A4AA979B9
:10FBA00012681278002A22D1132924D103223DE0C1
:10FBB000002D5ED02A88192A5DD1D97832784CE0A0
:10FBC0002C1E59D02A880024192A55D11C705C702B
:10FBD00052E0381C391C3A1CFAF7D0FC3C1C4BE0B4
:10FBE000042840D801F090FCD525313C2B00082991
:10FBF00042D104211970141C3EE0224A1268947804
:10FC0000002C0BD03178002908D05178022200292D
:10FC100000D104221A700022DA702DE03178002918
:10FC2000C4D051780122002900D104221A70012485
:10FC300022E0002D20D02A88192A1DD110E0002DA5
:10FC40001AD02A88192A17D1B0E7002D14D02A8893
:10FC5000192A11D10124D978327891420CD3A5E721
:10FC600000221A7008E0201C211C221CFAF786FCD6
:10FC700002E02C1C00E00024201CFEBDFE2F002012
:10FC8000F82F0020F42F002000300020F0B50026CF
:10FC9000CA4BB1B09C781F1CB44200D09AE104A8B2
:10FCA000FAF760FBB04203D0211C221CFAF766FC75
:10FCB000049E002E04D00122C14B00261A7089E157
:10FCC000311C18220EA801F0A9FC311C10220AA830
:10FCD00001F0A4FC311C072206A801F09FFCB94CDE
:10FCE00002ABDD1C207803A92A1CFFF743FE009419
:10FCF000002800D059E13878042837D801F00EFCEC
:10FD000003070D2E1B000020011C021C31E0012303
:10FD10002C783B71013CE4B22EE07B78FC78002B20
:10FD200003D12B78013B1C1BE4B201233B71FB7810
:10FD30000133FB7020E07B78FC78002B03D12B781B
:10FD4000013B1C1BE4B2002301223B71FB780192B2
:10FD50000133FB7063B2013313D14FE000233B71D9
:10FD6000994B1B681C78002C65D178E0301C311C45
:10FD7000321CFAF703FC71E0002263B201920133F6
:10FD80006CD02B7864B29C4235DC1CAD281CFDF78E
:10FD90009DFC0023AB70009B211C18786A2302ACE9
:10FDA00024AA1B192870FFF787FD0025002812D010
:10FDB00002AB03331B789D4200D3F6E0814B02ACCB
:10FDC00018786A2369B224AA1B19FFF775FD002869
:10FDD00001D00135ECE7002024A9FFF737FE041E0F
:10FDE00007D11CA806A9FDF77FFC002803D03C71B1
:10FDF00004E0061CEEE0019B002B2FD024210823F9
:10FE000002AA52182C21137002AA5218137014ABB4
:10FE10000A936C481CAB0AA90C93FDF747FA01241E
:10FE200000281CD0C1E0002800D0BEE0211CFFF754
:10FE30000DFE002807D0009B24AC1878211CFFF78A
:10FE40000BFE0828EFD108232370604B201C1A6892
:10FE50000C21F9F75FF9002800D0A6E000243B79D7
:10FE6000002B10D0012B00D09DE0302102AA5218A7
:10FE70001370042342217B7106AB0F93002302AA67
:10FE8000521813804BE0002C31D102AB03331B78A6
:10FE9000022B13D924AD281CFDF718FC8A22009BE5
:10FEA000211C187802ABD2182870FFF795FD0028A6
:10FEB0007BD1281CFDF754FA002876D10AAB1A79B9
:10FEC000002A74D11B7B002B71D1052338217B7153
:10FED000002302AA521840211370A02302AA52182C
:10FEE00042211380B42302AA5218138012E0042383
:10FEF00038217B71022302AA52184021137020235B
:10FF000002AA521842211380052302AA5218138014
:10FF10000AAB11933021002302AA521813707B7987
:10FF200005A82B490422009301F036FB08A8FFF72F
:10FF30008FFD002803D000210A1CFAF71FFB0020C8
:10FF400008A9FFF783FD002803D000210A1CFAF757
:10FF500015FB24AC0021201C302201F05FFB0223A2
:10FF600023706B4601251B78201CE370002105AB34
:10FF7000A57025826361FBF7E9F9002815D10EA869
:10FF8000FFF768FD002810D13B78BD70032B21D10D
:10FF9000072323700D4B201C1A680C21F9F7BAF8BF
:10FFA000002817D001E0032614E0061C12E0002010
:10FFB000011C021CFAF7E2FA87E7C046F82F00207E
:10FFC000FF2F0020FE2F0020F42F0020F02F002014
:10FFD000581D0200301C31B0F0BDC04610B503887A
:10FFE000112B09D0192B12D0102B1FD10022104B2E
:10FFF0009A705A701A7019E0FFF7A8FD002815D002
:020000022000DC
:10000000FFF744FE002811D000210A1C0CE0002458
:10001000074B9C70FFF79AFDA04207D0FFF736FE12
:10002000A04203D0211C221CFAF7A8FA10BDC0463A
:10003000F82F002037B50238012819D80D4B1A784F
:100040001D1C002A14D001A8FAF78CF9002803D04F
:1000500000210A1CFAF792FA019C002C08D12C709E
:10006000FFF714FE002803D0211C221CFAF786FAA1
:1000700037BDC046FF2F0020014B98787047C0461F
:10008000F82F0020FF23F0B585B001AC2371A371D8
:1000900063711A4BBC270D1C19780023184E7F0082
:1000A0008B4208DA3A1C5A43B218904201D12371AC
:1000B00001E00133F4E72379FF2B04D10020011C78
:1000C000021CFAF75BFA0023E3712B780195042BED
:1000D00008D1EB79A371AB796371EB68A3606B898D
:1000E000E37105E0072B03D1EB79A371AB79637161
:1000F000044B201C1B68984705B0F0BD043000205D
:100100000C3000200830002070B50F240126027842
:100110004378A243324385782240002901D0302120
:1001200000E02021A543A34333432E432340344022
:100130000A430B430C4302704370847070BD00008F
:10014000F0B5066887B00723002E6DD04468002CF8
:100150006AD0018A002967D08568002D64D0C26802
:10016000002A61D00423232A5ED9314B314F1E600F
:10017000314B324E1C60324B324C1A800023324AD3
:100180002560324D11803B7033702B70837C9370EF
:10019000C37CD370037D1079033B591E8B412C49DE
:1001A000DBB20B700F21023308401B010343DBB2AB
:1001B0008B4301210B4313710023FF21537102A8CC
:1001C000082201F02BFA206802A9082201F0BAF9EE
:1001D000002802D03B7801333B7004A8FF2108229D
:1001E00001F01CFA00235F1C2368F800181804A90A
:1001F000082201F0A7F9002802D0337801333370C8
:100200003B1E032BEFD1FF21042201A801F006FAC7
:10021000206801A92030042201F094F900239842BB
:1002200002D02A7801322A70181C07B0F0BDC046EF
:1002300008300020043000208C310020883100205C
:10024000983100208431002092310020903100202C
:1002500091310020F0B587B001900293019B0C1CF6
:1002600003920720002B5DD000295BD0029B002B5E
:1002700058D000252C4F2D4E3B789D4211DA326824
:10028000EB00D3189A88A24209D119680198221C60
:1002900001F058F9002802D1029B1D7042E001359F
:1002A000EAE737683D1C2435012B08D1BE88013EA2
:1002B000F217920F9619B6100136B600AD191C4907
:1002C0002A190988042079188A422BD86946097BA3
:1002D00004AAD17193719480029A04A91370DB006F
:1002E000F8180222049500F0A1FF0F4B0E4A1B786C
:1002F000013C013313708022520513695169A41027
:100300004B4301340198A20082189A4204D900207C
:10031000011C021CFAF732F9A2B2281C019900F064
:1003200085FF002007B0F0BD04300020843100209C
:1003300098310020F0B587B001930CAB1B78051CF9
:100340000293364B0E1C1B78171C0720AB4263D957
:100350000D9B002B60D0324A324B117800221B6873
:10036000C90059188B4209D0187AA84204D1587A8A
:10037000B04201D10132D2B20833F3E70D9B002124
:100380001A7004A8082201F049F904AB1D70DF704F
:100390005E700D9B04AA1B78214C9370131C6A4657
:1003A000127921781A716A46127A03945A711D4B98
:1003B0001A680023101C08308B421DDA0478AC4206
:1003C00017D1C478BC4214D10479A446019CA44539
:1003D0000FD14479A446029CA4450AD14478B44282
:1003E00007D10133DB00D3189B78FF2B04D00D9A83
:1003F00010E001330830DFE7042002290CD8481C44
:10040000C000101804A9022200F010FF039B039AF9
:100410001B7801330020137007B0F0BD04300020BA
:100420008831002084310020F0B5B1B018210022BD
:100430000CA801F0F3F81821002212A801F0EEF840
:1004400018A81821002201F0E9F800259F4B1B781D
:100450009D4200DB34E19E4B01221F68EB00FB183C
:10046000DC790026231C13400493069363083C1C8C
:10047000134005930834039602960196954B1B781A
:100480009E425CDA2378AB4256D16378012B19D1B6
:10049000019A6179D2000CA81152217980188170DB
:1004A0006278C270E178C27919409A438A4B0A4354
:1004B000C27119780430FFF727FE019B0133DBB2CC
:1004C000019339E0022B1AD10121029B6279DB00F2
:1004D00012A81A522279C01882706378C370E27829
:1004E000C3790A408B431343C3717B4B04301978A3
:1004F000FFF70AFE029B0133DBB202931CE0032BE1
:1005000000D0DFE00121039B6279DB0018A81A52BA
:100510002279C01882706378C370E278C3790A4088
:100520008B431343C3716C4B04301978FFF7ECFD18
:10053000039B0133DBB20393013608349EE70024AA
:10054000664B261C1B7809AA00933B1C203300999C
:100550008C4210DA1978A9420AD101200790684626
:10056000B100007F5718B8705F8801368F52F6B21D
:1005700001340433EBE71EAC201C0021482201F0BB
:100580004DF8574B524A1E93564B12681B6808A9E8
:1005900063606B461B7E2AA823726B461B7D6372C9
:1005A0006B461B79A3720CABE3606B461B7A23741A
:1005B00012AB63616B461B7B237618ABE361EB00E8
:1005C000D3189A88A2841B6808AA236209ABA36285
:1005D0005F239B188E22DE77002352181370424946
:1005E0000622A36300F0D8FF3B4B012619780F23A6
:1005F0002DA8027830249A4332431A40002900D1B2
:10060000202422430270952208A8121810789843DB
:10061000304303401C4314709622002008AC12198A
:10062000107048424841032297240F230126121AD2
:1006300008A824182078120118401043C0B298432B
:100640003043207029A804781C401443E4B29C4332
:10065000344385220470002008AC12191070049AEB
:10066000824219D09E200019027830249A433243E6
:100670001A40002900D12024224302709F2208A89A
:10068000121810789843304303409B201C4308AB5A
:100690001470C018FFF738FD059B002B04D00E4BDB
:1006A0002EA81978FFF730FDBC20400068430F4B9F
:1006B0001EA91818FBF77CFF002804D10135C5E6F8
:1006C000002000E0032031B0F0BDC046043000201F
:1006D00084310020883100209131002090310020A9
:1006E000850002008C310020923100200C30002067
:1006F000F8B5061C0024074D074F2B789C4208D202
:10070000BC2040006043311C3818FBF70DFE01345B
:10071000F3E7F8BD043000200C30002038B5BC24CD
:10072000151C64006043034A10189AB22B1CFCF796
:1007300001FA38BD0C30002008B5084B021C1B78AC
:100740000821002B08D0A72305485B00C35A002BC3
:1007500002D0FCF729FA011C081C08BD0430002057
:100760000C30002013B50C4A031C12780820002A14
:1007700010D0AF22094C5200A25A002A0AD00122FE
:10078000002019789A569B78009001905BB2201C4B
:10079000FCF73AFA16BDC046043000200C300020A9
:1007A000F0B500240226144B251C1A68134B111CAB
:1007B0001878B446131CC000101883420AD00127D1
:1007C000DE793E4200D03D1C67463E4200D0012407
:1007D0000833F2E700200A4B1B78DB00D31899425C
:1007E00006D04A7A0831013A564272418018F6E73B
:1007F00040190019F0BDC0468431002004300020AB
:1008000088310020F7B5FDF717FA031E4CD1191CEB
:100810001A1CFDF799FB01A8FDF748FB002808D03A
:10082000019B180AC0B200F031FD019BD8B200F064
:100830002DFD0024251C271CFDF7C0FA6B46061C65
:10084000D81C00F009FD0028F6D06B46DB78002D9F
:1008500003D11C02371C0125EEE73A1C13329642E5
:1008600002D91C02371CE7E71C433F23210AA208D8
:1008700019401A400323A00B80B22340032B01D15F
:1008800001235B42FDF760FB01A8FDF70FFB00258C
:10089000A842D1D0019B180AC0B200F0F7FC019B1E
:1008A000D8B200F0F3FCC7E701204042FEBD0000D3
:1008B000012310B509495C5C0A1C84420DD0013348
:1008C000072BF8D10023D1184C780133002C02D12A
:1008D0004870D37101E0062BF5D110BDB031002076
:1008E0002FDF704732DF704736DF704737DF7047E2
:1008F00012DF7047002008B5011C054AF8F70AFC12
:10090000002803D000210A1CF9F738FE08BDC046B4
:10091000F50B020008B504490A2200F013FE434219
:100920005841C0B208BDC046D0310020072301287D
:1009300002D8024B18700023181C7047BA310020EF
:1009400070B5084E08203578002D09D10124FDF737
:10095000FBFC201C3470FDF71BFD281C024B1C7097
:1009600070BDC0469D3100209B31002010B5054C64
:100970002378002B05D0044B1868F9F771F8002391
:10098000237010BDC4310020C03100200723F0B512
:1009900085B00290434944485A1E0E1C002A04D0D8
:1009A000023BCC5CC454131CF6E7404C404D23780A
:1009B000081C211C2B70FDF747FD0194071E01D177
:1009C00000206DE03B4B1A680393511E1960002A0A
:1009D00001DD002207E0FEF749FE0028F9D0364B82
:1009E0001A78531E9A41019B29781B7800918B42FB
:1009F0000BD10B1C2C49013B04D3F45C585C8442A2
:100A0000F9D002E0002ADBD0002700252B4C6570CE
:100A1000A570E57025716571A5712570E571009B64
:100A20009D4215DA019B1A78002393420EDA1E4884
:100A3000F15C285C884207D1031C2033DBB2072B12
:100A400004D9FFF735FF01E00133EEE70135E6E7B2
:100A50000025019B1B789D4213DA705D031C203337
:100A6000DBB2072B07D80122E0388240101C237824
:100A70001843207003E0002801D0FFF719FF01356B
:100A8000E7E7601C2178E279FDF76CFD029B20729C
:100A90001C600323002F00D01A230120039A136047
:100AA00005B0F0BDA8310020A03100209C3100200D
:100AB0009A31002020200020BA310020B0310020DF
:100AC000F0B5374B85B01B78002B67D0FDF790FC55
:100AD000344C051E12D1344B34481A680A21F8F7F9
:100AE00019FB002803D0291C2A1CF9F747FDFFF742
:100AF0003DFF0020FDF74CFC00234EE02378002B47
:100B00004CD103A8FFF742FF002847D0284B1B78A1
:100B1000002B2FD103990A26CA79081C0192302292
:100B200008279446421A019DD2B2AA4221D24278A5
:100B3000151C1E3D092D09D85D1CCB18272A01D193
:100B4000624600E013325A702B1C10E0151F192D5D
:100B500003D85D32CD186A7008E02A2A02D1CA187B
:100B6000577003E0282A02D1CA18567001330130A9
:100B7000D8E7CB710C4B03981B680A219847039860
:100B8000FFF7C8FE002809D0FFF7F0FE1A22094B34
:100B900001201A60FDF7FCFB0123237005B0F0BDB6
:100BA0009D3100209B310020BC310020C631002047
:100BB000BA3100202020002070B50C4B1C781E1C80
:100BC000002C11D1051C201CFFF77AFF084B291CB3
:100BD0001868221CF8F7EEFE002803D0211C221C06
:100BE000F9F7CCFC01233370002070BDC431002024
:100BF000C031002008B5074B1B78002B05D0002022
:100C0000FDF7C6FB0022044B1A70F6204000FFF7E8
:100C1000D3FF08BD9D3100209B31002070B5072413
:100C200001283AD8002938D01D4E08243578002DE7
:100C300033D11C4B062218701B4B1C4819601C4BEF
:100C4000291C1D701B4B1D7000F0E8FC291C06229E
:100C5000194800F0E3FC291C0A22184800F0DEFCC9
:100C6000291C0125164C0A22201C00F0D7FC15482F
:100C7000291C154A6572F8F777FE041E0DD1FDF7A1
:100C8000FDFC041E09D104201049FDF72DFD041EB2
:100C900003D1211CFFF7AEFF3570201C70BDC0468C
:100CA000C5310020BA310020BC310020A83100201D
:100CB0009C3100209A310020A0310020D03100204A
:100CC000C6310020C0310020C10A0200F508020030
:100CD00008B5FDF78DFB08BD73B56B4600249E1D5E
:100CE000DD1D301C34702C70FFF702FEA04203D0D3
:100CF000211C221CF9F742FC3378012B0ED1281C51
:100D0000FFF7F2FDFFF732FE0620FFF7E9FD0620B0
:100D1000FFF7E8FD2878FFF7E9FD06E04023074AE2
:100D20000749D367C02252008B50FDF761FB0028B2
:100D300001D0FDF767FB012076BDC04604E100E06D
:100D400000E100E03CDF704749DF70474ADF704751
:100D50004BDF704748DF704712DF704713B56B46B3
:100D6000DC1D0023201C2370FFF7F6FF2378002BE7
:100D700004D180230122DB055A6001E0FFF7E6FF82
:100D800013BD0000F0B580260124214BF605F5586F
:100D900085B02540019338D102ABDF1C0090381C90
:100DA000DD70FFF7D9FF3A78002A21D1194B5A603C
:100DB0003460009A002A28D0221C5D68002D24D1BE
:100DC000E12080000138C046C046C046C046C0464B
:100DD000C046C046C046C046C046C046C046F1D127
:100DE000019971582142E8D18021C9050A60E4E7E0
:100DF000FFF7AAFF009B002B07D00395039B002B56
:100E000003D103A8FFF7A4FFF8E705B0F0BDC04683
:100E10000C040000FC00004070B5C223802518229D
:100E2000ED059B00EA5000230126284C284A236147
:100E30006361AA58324203D1301CFFF7A3FF331C71
:100E400001222A612269002AFCD000211F4A116177
:100E50008B4201D0FFF782FF8023C1221821DB05DE
:100E6000920099501B4A20201168A722D200995065
:100E70000138C046C046C046C046C046C046C0460F
:100E8000C046C046C046C046C046F1D10121202020
:100E900099610138C046C046C046C046C046C046FB
:100EA000C046C046C046C046C046C046F1D1C0207C
:100EB000FF24094A596180001358A343C0242343E7
:100EC0001350C0235B00D150116070BDFC00004086
:100ED0000C0400002C20002000E100E037B5214A7E
:100EE00021491368096801331360151C01AC002007
:100EF0008B4208D1012323701C4B60701A68201CA0
:100F00000221F8F707F91A4B2A681B689A4209D39D
:100F10000023237001236370144B201C1A680221E4
:100F2000F8F7F8F8002803D000210A1CF9F726FB8F
:100F30000023201C2370FFF70FFF217800290FD119
:100F40000C4B0D4C1A68207801321A60002802D030
:100F50001960217004E0092A02D91860FFF75CFFCC
:100F600037BDC0460C32002024200020E031002094
:100F700028200020FC3100200032002070B580269F
:100F80002C4CF6056369002B19D0002320206361E7
:100F90000138C046C046C046C046C046C046C046EE
:100FA000C046C046C046C046C046F1D10125756165
:100FB000281CFFF7E7FE204BB56735611D702369DC
:100FC000002B35D020200138C046C046C046C04660
:100FD000C046C046C046C046C046C046C046C046E1
:100FE000F1D120200138C046C046C046C046C046A8
:100FF000C046C046C046C046C046C046C046F1D105
:1010000020200138C046C046C046C046C046C04643
:10101000C046C046C046C046C046C046F1D10022C8
:10102000044B1A61FFF79AFE80230122DB05DA6781
:1010300070BDC046FC0000400032002037B56B4652
:10104000DD1D00232B70984201D107244CE00029BC
:10105000FBD0264A041C1160011C254A183113607C
:10106000026A244B1A60244B426A24481A60082200
:1010700000F092FA18222248211C00F08DFAA36A8F
:101080005A1E7E2AE1D81F4A281C1360FFF764FE0F
:101090002B78002B16D180228323D205DB00D15878
:1010A00080235B020B400BD1A321C90053500123C5
:1010B0009360154A9368002BFCD00022124B9A6073
:1010C000FFF7AAFE114D0121281C114AF8F74CFC2C
:1010D000041E09D10120FFF755FE8021221C28683B
:1010E0000902F8F767FC041C201C3EBDE03100201B
:1010F0000C32002028200020242000200432002070
:10110000E43100202C200020FC000040DC310020D5
:10111000DD0E02000022024B1A60024B186070477D
:101120000C3200202820002008B5FFF713FE02280B
:1011300003D120BF40BF20BF06E0002804D000201C
:10114000011C021CF9F71AFA08BD000038B500248A
:10115000064D2B789C4205DAA300EB185B68984794
:101160000134F6E7FFF7FAFD38BDC046043200202F
:10117000F7B56B4600240126DD1D114F2C703B781E
:101180009C420ADAA300FB185B6801209847431EC3
:101190009841404206400134F1E7002E0ED0281C51
:1011A000FFF7DAFD2B78002B02D0FFF7CBFD05E02F
:1011B000A02380220121DB00D205D150F7BDC0461B
:1011C000E4310020002008B5024B1860FFF7DAFD7B
:1011D00008BDC0460C32002048DF704770B5041CC3
:1011E0000D1C0F4E3378002B02D0FFF7F5FFF9E707
:1011F000012180260B4B0C4AF6009950802099590A
:10120000C0000029FAD0256019580029FCD0002020
:10121000044988508021C9005A58002AFCD070BD6A
:101220001032002000E001400405000070B5051CEC
:101230000E1C92008418A54205D0281C02CEFFF790
:10124000CDFF0435F7E7002070BD0000014B18709A
:101250007047C0461232002010B5094B1B78002B96
:101260000CD008490022CC68012C06D1CA60A32208
:101270000549D2008A58027000E0131C181C10BDEA
:1012800011320020FC20004000200040074B1B785A
:10129000002B09D0064A074BD050074A136A012B8E
:1012A000FCD10022044B1A627047C0461132002064
:1012B000002000401C050000FC20004010B5094B38
:1012C000041C1B780078002B0AD0074B1B78002BDE
:1012D00006D10134002803D0FFF7D8FF2078F8E7C3
:1012E00010BDC04611320020123200201FB5064B3F
:1012F0001B78002B06D001A9102200F059FA01A892
:10130000FFF7DCFF05B000BD113200201FB5064B12
:101310001B78002B06D001A90A2200F049FA01A887
:10132000FFF7CCFF05B000BD11320020F7B59C4699
:1013300008AB1B782B4C01932B4B1D682B4B9D420C
:1013400004D0A0230022DB00E2504AE00E1CA025BE
:101350000323C136FF36ED05B600735166460027FC
:10136000C136FF36B6007751214EA151664621495C
:1013700066500199B94212D0011CC131FF31890078
:101380004B51131CC133FF339B005F51A223DB0081
:10139000E250A1230122DB00E050174BE250174A34
:1013A000174B0125E250A0230422DB00E250FA2073
:1013B0000022144BA56080002560DA600138C04629
:1013C000C046C046C046C046C046C046C046C046ED
:1013D000C046C046C046F1D10B48FFF76FFF0B4B2C
:1013E0001D70F7BD00200040009703005541525486
:1013F0000C050000140500006C05000000E0D7019A
:1014000024050000FC2000405C1D02001132002079
:1014100003210F4802680A4302600E4802680A432B
:1014200002600D490D4A0E4B9B1A03DD043BC85860
:10143000D050FBDC00200B490B4A0860043191427C
:10144000FBDB0A4885460A4880470A4800470000F7
:101450002405004054050040A41D02000020002087
:1014600030200020302000205C320020004000208E
:1014700015E1010001AE0100FEE7FEE7FEE7FEE731
:10148000FEE7FEE7002804DA4042002904DA494278
:1014900020E000291EDA494200B500F01BF8404266
:1014A00000BD00280EDA4042002905DA494200B5A5
:1014B00000F010F8494200BD00B500F00BF84042C2
:1014C000494200BD002905DA494200B500F002F8A2
:1014D000404200BD002900D114E0012200238842CF
:1014E00006D9003104D45200490001D48842FAD808
:1014F000884201D3401A134349085208F8D10146E3
:1015000018467047FFF7FEFF02B4714649084900CC
:10151000095649008E4402BC7047C04602B4714669
:1015200049084900095C49008E4402BC7047C04626
:1015300003B47146490840004900095A49008E44E5
:1015400003BC704730B5032A20D9031C0B439B070B
:1015500013D004780D784B1C8A18AC4206D018E0E2
:101560000133591E04780D78AC4212D101309342F8
:10157000F6D1002030BC02BC084703680C68A342C7
:1015800004D1043A04300431032AF6D8002AE0D109
:10159000EFE7601BEEE7C046F0B50F2A36D9031C13
:1015A0000B439B0736D1151C031C103D2D0901353B
:1015B0002D014C190E681E604E685E608E681031F9
:1015C0009E600E1F376810331E1F3760A142F1D195
:1015D0000F2345191340032B1ED90021043B9B0800
:1015E00001339B0066586E5004319942FAD10323AF
:1015F0006D181A406118002A05D00023CC5CEC5409
:1016000001339342FAD1F0BC02BC0847051C002A02
:10161000F3D1F8E7051CF0E71A1CF8E770B583076B
:1016200042D0541E002A3CD00D062D0E031C03266A
:1016300003E0621E002C34D0141C01335A1E1570B6
:101640003342F6D1032C23D9FF220A4015022A4344
:1016500015042A430F2C2AD9251C103D2D090135CC
:101660002D015D191A605A609A6010331E1F326096
:101670009D42F7D10F263440032C09D9231F9B0824
:1016800001339B00EB1804C5AB42FCD1032214408C
:10169000002C06D009061C19090E19700133A3424B
:1016A000FBD170BC02BC0847141C031CCAE71D1CFC
:1016B000E4E7C04610B5830729D00378002B28D073
:1016C000031C032102E01A78002A1CD001330B42CC
:1016D000F9D11968104A114C8A188A4322420FD155
:1016E000043319680C4A8A188A43224208D1043309
:1016F0001968094A8A188A432242F1D000E001336E
:101700001A78002AFBD1181A10BC02BC0847031C27
:10171000DFE70020F8E7C046FFFEFEFE8080808005
:10172000F0B5574645464E46E0B48AB090466A4604
:101730001E4B0D1C061C13CB13C213CB13C213CBB1
:1017400013C21B7813704346023BEA462F1C002449
:10175000222B01D926E04C46631C301C4146994699
:10176000FFF7B8FE53465B5C301C3B704146FFF709
:10177000B1FE0137061EEED14B46E8540023002C83
:1017800007D0EA5C295DE9542A550133013CA342A4
:10179000F7DB281C0AB01CBC90469946A246F0BC58
:1017A00002BC08472C700020F4E7C046741D0200FC
:1017B00008B5FFF7B5FF08BC02BC0847F8B5C0463E
:1017C000F8BC08BC9E467047F8B5C046F8BC08BCDB
:1017D0009E4670470D0A4164647220000D0A426102
:1017E00074746572792070657263656E74206368C5
:1017F0006172676520000D0A456E746572696E67D7
:101800002042696E617279206D6F646520286E6F69
:10181000206D6F726520737472696E677320666FD6
:101820007220796F75290D0A000D0A61202D206143
:101830006464726573732C2062202D20626174745D
:101840006572792C2064202D2064656275672061A3
:101850006464726573732C2068202D2068656C7039
:101860002C2069202D2049442C000D0A6B202D20AE
:10187000746F67676C65206B65796C6F6767696EFD
:10188000672C206C202D206C696420737461746552
:101890002C2072202D20726573657420656E616244
:1018A0006C652C2076202D2076657273696F6E0D25
:1018B0000A000D0A494420006B65797374726F6BDE
:1018C00065206C6F6767696E672000646973616289
:1018D0006C65640D0A00656E61626C65640D0A00DA
:1018E0000D0A4C696420006E6F742000707265737D
:1018F000656E7400526573657420656E61626C6517
:10190000642C20686F6C64207265736574206C6F42
:101910007720746F2065786974206465627567202C
:101920006D6F64652E0D0A000D0A56657273696F3E
:101930006E2000204275696C74206F6E2000446533
:101940006320313120323031350020617420003184
:10195000373A30323A3434002070726573736564FC
:101960000D0A002121212121204150505F45525272
:101970004F525F48414E444C4552202121212120A5
:101980006572726F725F636F6465203D203078000E
:10199000696E2000204020004520000D0A5570642B
:1019A000617465210D0A00504149520D0A007061B1
:1019B00069720D0A004C6964206E6F742070726544
:1019C00073656E740D0A004D6F64696669657220F7
:1019D000427974653A20307800204E756D204B6551
:1019E00079733A2000205363616E20436F646573FE
:1019F0002028686578293A200062460D0A0050695F
:101A000078656C2043204B6579626F617264004792
:101A10006F6F676C6500302E3135313231300045E3
:101A200072726F72200020747279696E6720746F11
:101A3000200055706461746520746865206C65765B
:101A4000656C20746F2000436F6E0D0A004665615F
:101A50007475726520004F75747075742040002095
:101A600064617461200020696E6465782000206CD8
:101A7000656E2000206964782000436F6E6E2055EB
:101A800070646174653A20696E74657276616C2069
:101A9000002C20736C617665206C6174656E6379CF
:101AA00020002C207375706572766973696F6E20E3
:101AB00074696D656F75742000416476420D0A008B
:101AC00041646472204368616E676564200D0A009A
:101AD00057616974696E6720666F722070617373F5
:101AE0006B65790D0A004F4F424B65792052657145
:101AF000210D0A00506173736B657920726563650F
:101B0000697665640D0A0052656164205265712032
:101B100000446973636F6E6E0D0A004469736162FD
:101B20006C65640D0A0041647665727469736520A2
:101B3000616761696E0D0A00506F776572204F66AC
:101B4000660D0A0054696D656F75740D0A00537453
:101B5000617274204446550D0A0045767420005287
:101B60006573657420526561736F6E203D20307817
:101B700000636F6D7320696E6974200D0A007077C1
:101B80007220696E69740D0A0072656164793E2085
:101B90000000000005010906A101050719E029E779
:101BA00015002501750195088102950175088101CF
:101BB000950675081500256505071900296581003A
:101BC000950575010508190129059102950175030F
:101BD00091010905150026FF0075089502B102C0A4
:101BE00077696C6C2074727920616761696E206C12
:101BF000617465720D0A006D5F7570646174655F74
:101C0000636F756E742000706172616D65746572CA
:101C1000206572726F7220636F646520006469735F
:101C2000636F6E6E656374206572726F7220636F8E
:101C30006465200023D1BCEA5F782315DEEF121221
:101C400000000000C7CC010069CE0100CBCC010030
:101C500025CF0100CFCC01002DCF0100D3CC010056
:101C600061CF0100D7CC01009DCD0100DBCC01008C
:101C700061CE0100FFFFFFFFFFC1FBE84C90728BBC
:101C8000E7B3518963AB232302841872AA612F3B07
:101C900051A8E53749FBC9CA0C18532CFD000000B8
:101CA0000000E00000000000E3002B00041D1E14F3
:101CB0000000000007062008050A1722091921154F
:101CC00000000000161B1F1A000000000E36250C35
:101CD000110B1C230D1024180000000000E100E58A
:101CE0002E34002D33382713000000000F37261242
:101CF000E60000000000E200002A0000282C5152FB
:101D00000000000000004F50020A07050309081BED
:101D100012100C0F0B0000000D0A42617474657202
:101D20007920766F6C7461676520002075560D0A06
:101D3000000000006456463C090600000B79410093
:101D4000C06A3E00AEAF3B00B9943A00B8A7370076
:101D5000EB113700C29F3300121801000D0A5541E4
:101D6000525420696E697469616C697A65640D0A00
:101D70000000000030313233343536373839616293
:101D8000636465666768696A6B6C6D6E6F707172AB
:101D9000737475767778797A0000000074F6FF7FA7
:101DA000010000004B4200000000000000000000A5
:101DB000000000000000000000800040080000005B
:101DC000040000001A000000FFFFFFFFFFFFFFFFFD
:101DD00020000000FFFFFFFFFFFFFFFFFFFFFFFFEF
:101DE000FFFFFFFFFFFFFFFFFFFFFFFFFFFFFFFF03
:101DF000FFFFFFFFFFFFFFFFFFFFFFFFFFFFFFFFF3
:101E0000FFFFFFFFFFFFFFFFFFFFFFFFFFFFFFFFE2
:101E1000FFFFFFFFFFFFFFFFFFFFFFFFFFFFFFFFD2
:108C000056623253030000004801000038000000A3
:108C100010000000480000000001000000FC0000FF
:108C200003000200419A32EEE5DBBCC148D6431393
:108C30008799B21B5DA65DFF4861646F6B656E200E
:108C400052656C6561736500631966EC911A1625AF
:108C50005B6798BE1EB9A35ADAEEE7F939C8E9AEE8
:108C60006DEFF4A8AC2CD775851B3FD387E18963E2
:108C70002C8F3398FBBC73ADB500592AAAA889473D
:108C80006171C124D0A820DC6AA05594A0315C1881
:108C90003CDC0D033749150EF8C5E15BB507268BA3
:108CA000310BB71C4BBC48BA26F59A4599F9803F61
:108CB0008B4EB8C02FD6DBE301237EC49562A5504E
:108CC0005EC163F0FC54B10CC96C28DE2E46CC901A
:108CD0004E491856EBDFD34AD999E632589F958210
:108CE000227244F8D9364CC97DBB3B471141F7DEAF
:108CF000A398B5E82A9C61FACF3DB02A1A60C0EF6C
:108D00006311AAEC7F33FA21378A5C1E55EFE0220B
:108D1000890D7771C92C5684556974ED50F7650B30
:108D20004A807280FE5528DC10E32BC633B009D18F
:108D30005F0339B903643D70486138FD1D3C96629C
:108D40006D2AFE7A5E2EC2DEFFFFFFFFFFFFFFFFF0
:108D5000FFFFFFFFFFFFFFFFFFFFFFFFFFFFFFFF23
:108D6000FFFFFFFFFFFFFFFFFFFFFFFFFFFFFFFF13
:108D7000FFFFFFFFFFFFFFFFFFFFFFFFFFFFFFFF03
:108D8000FFFFFFFFFFFFFFFFFFFFFFFFFFFFFFFFF3
:00000001FF
